:0200000480007A
:10000000B72F0000938F0F8073900F3015A8130047
:100010000000130000001300000013000000130094
:100020000000130000001300000013000000130084
:100030000000130000001300000013000000010086
:10004000970200009382020C73905230814001416C
:100050008141014281420143814301448144014580
:100060008145014681460147814701488148014950
:100070008149014A814A014B814B014C814C014D20
:10008000814D014E814E014F814F971102009381A6
:1000900021D4170502001305E556979503009385B3
:1000A000257601461122170502001305E54997053B
:1000B0000200938585510146C52817A50300130545
:1000C000657497B503009385A57337B6ABAB13067C
:1000D000B6BAD92817B103001301C172EF60205FCF
:1000E000860293D21200F512638802008242110147
:1000F0006F00001073002030824211017300203025
:10010000711116C0F3222034E3CC02FC82421101AB
:10011000130141F806C20AC40EC612C816CA1ACC88
:100120001ECE22D026D22AD42ED632D836DA3ADCC7
:100130003EDEC2C0C6C2CAC4CEC6D2C8D6CADACC97
:10014000DECEE2D0E6D2EAD4EED6F2D8F6DAFADCA7
:10015000FEDE73252034F32510340A8601A07310C7
:10016000153492402241B2414242D2426243F243AC
:10017000025492542255B2554256D2566257F25703
:10018000064896482649B649464AD64A664BF64B33
:10019000065C965C265DB65D465ED65E665FF65F83
:1001A0001301C1077300203010C16374B50011053D
:1001B000E5BF828000000000000000000000000099
:1001C000000000000000000000000000000000002F
:1001D000000000000000000000000000000000001F
:1001E000000000000000000000000000000000000F
:1001F000197106C00AC20EC412C616C81ACA1ECC8D
:1002000022CE26D02AD22ED432D636D83ADA3EDCC6
:1002100042DEC6C0CAC2CEC4D2C6D6C8DACADECC96
:10022000E2CEE6D0EAD2EED4F2D6F6D8FADAFEDCA6
:100230009702020083A2823423A02200F32210340A
:1002400096DEEF00002B170102000321213302414B
:10025000F65273901234B72200009382028873A082
:10026000023082403242C2425243E24372448254DC
:100270001255A2553256C2565257E2577258864806
:100280001649A649364AC64A564BE64B764C865C1A
:10029000165DA65D365EC65E565FE65F0961730059
:1002A0002030970202009382E23523A0120023A29D
:1002B000220023A4320023A6420023A8520023AA2E
:1002C000620023AC720023AE820023A0920223A21C
:1002D000A20223A4B20223A6C20223A8D20223AA06
:1002E000E20223ACF20223AE020323A0120523A2F2
:1002F000220523A4320523A6420523A8520523AADA
:10030000620523AC720523AE820523A0920723A2C7
:10031000A20723A4B20723A6C20723A8D20723AAB1
:10032000E20723ACF207EF40D0551701020003218A
:10033000E1240241F65273901234B72200009382F6
:10034000028873A0023082403242C2425243E243EA
:10035000724482541255A2553256C2565257E25731
:10036000725886481649A649364AC64A564BE64B45
:10037000764C865C165DA65D365EC65E565FE65FB1
:10038000096173002030970202009382A22783A0A4
:10039000020003A1420083A1820003A2C20083A243
:1003A000020103A3420183A3820103A4C20183A427
:1003B000020203A5420283A5820203A6C20283A60B
:1003C000020303A7420383A7820303A8C20383A8EF
:1003D000020403A9420483A9820403AAC20483AAD3
:1003E000020503AB420583AB820503ACC20583ACB7
:1003F000020603AD420683AD820603AEC20683AE9B
:10040000020703AFC20983AF820782807370043092
:10041000197106C00AC20EC412C616C81ACA1ECC6A
:1004200022CE26D02AD22ED432D636D83ADA3EDCA4
:1004300042DEC6C0CAC2CEC4D2C6D6C8DACADECC74
:10044000E2CEE6D0EAD2EED4F2D6F6D8FADAFEDC84
:100450009702020083A2821223A0220086DEEF20F0
:10046000205D17010200032161110241F6527390D1
:100470001234B72200009382028873A002308240B7
:100480003242C2425243E243724482541255A25550
:100490003256C2565257E257725886481649A649F4
:1004A000364AC64A564BE64B764C865C165DA65DD0
:1004B000365EC65E565FE65F09617300203073707A
:1004C000043001A07310453082807325403073F0F2
:1004D00043308280970700009387A7FE232EB5FE46
:1004E0002322C5FA232635F82320F5F8130505F84D
:1004F0008280411106C6EF403036EF10103B01E517
:10050000B24041018280B24041016F2060529307A6
:1005100085007D575CC118C55CC51CC9232005003A
:1005200082802328050082805C41DCC1984798C501
:1005300098474CC38CC788C91C4185071CC1828061
:100540009041FD57130785006314F60039A83E87D4
:100550005C439443E37DD6FEDCC18CC798C54CC395
:1005600088C91C4185071CC1828018495C43EDB7CE
:10057000584114451C4914C71845544154C3D84325
:100580006314A7001845D8C32328050088437D15A8
:1005900088C382803041AE8701CE4C455841B29528
:1005A0004CC563E4E5000C414CC53E856F30704F8F
:1005B0008280411122C406C62A8426C2EF20F04060
:1005C0003C44635BF0025C5085CB9304440209A871
:1005D0003C44FD173CC43C446350F0025C5089CF5E
:1005E0002685EF2010076DD5EF20F0263C44FD173F
:1005F0003CC43C44E344F0FEFD573CC4EF20303F94
:10060000EF20B03C7C40635BF0021C4885CB930438
:10061000040109A87C40FD177CC07C406350F002B7
:100620001C4889CF2685EF20D0026DD5EF20B0225F
:100630007C40FD177CC07C40E344F0FEFD577CC04D
:100640002244B240924441016F20703A29CD0111F9
:1006500022CC2A8406CE26CA4AC84EC62E89EF204E
:10066000D03624404C5C832904002685EF50D06F9F
:100670007D57232C0402B3079540CE974E9578C042
:1006800048C0232434015CC438C4631109021C48E7
:100690008DE7EF20D035F2406244D2444249B2495E
:1006A0000545056182807370043001A013050401C3
:1006B000B93D13054402A13DE9BF13050401EF2034
:1006C00040798547E317F5FC9133E1B701E5737095
:1006D000043001A0011126CA4AC84EC606CE22CC5B
:1006E000AA842E89B289A5C9EF5010681305550553
:1006F000EF30F0222A8435C5930745051CC144DC40
:1007000023202405EF20702C24404C5C0329040096
:100710002685EF507065FD56232C0402B3079540E3
:100720003307A900CA9774C058C05CC434C4130509
:10073000040123242401E13B13054402C93BEF20BB
:10074000102B230834052285F2406244D2444249EA
:10075000B2490561828013054005EF30501C2A84A0
:1007600001E57370043001A000C051BF01E5737052
:10077000043001A06375B5007370043001A041110D
:1007800022C409462E84814506C6893711C500DD7D
:10079000B2402244410182807370043001A05D7137
:1007A00086C6A2C4A6C2CAC04EDE52DC56DA5AD8E9
:1007B0005ED632C6630A051C6382051C89476399AD
:1007C000F600585D85476305F7007370043001A09B
:1007D0003689AE842A84EF20900A11E5B24781C79A
:1007E0007370043001A0EF20501E185C5C5C014B5C
:1007F000894BFD59130A0401930A44026365F70CFF
:1008000063077919B2476381072463150B00280831
:10081000EF204077EF20B01DEF10E07FEF20F01ABF
:100820007C4063943701232204043C4463943701E1
:1008300023240404EF20B01B6C002808EF20A076CE
:10084000631E051EEF207018185C5C5C630CF70AD1
:10085000EF20F019EF2070173C44634FF00039A8E7
:100860005685EF20005F19C1EF20E07E3C44FD1764
:100870003CC43C446354F0005C50FDF32324340535
:10088000EF20F016EF2070147C40634FF00039A881
:100890005285EF20005C19C1EF20E07B7C40FD1702
:1008A0007CC07C406354F0001C48FDF323223405D7
:1008B000EF20F013EF10301B054BEF201011185CE8
:1008C0005C5CE37FF7F230406305060C631F09129E
:1008D0000844A685EF30F01C1C4434405840B697BD
:1008E0001CC463EAE70A1C5C14405850850714C412
:1008F0001CDC5DC713054402EF20A055854763113A
:10090000F50AC9A8EF20B00EB2455285EF20203677
:10091000EF20B00B3C44634FF00039A85685EF2020
:10092000405319C1EF2020733C44FD173CC43C44A4
:100930006354F0005C50FDF323243405EF20300BAA
:10094000EF20B0087C40634FF00039A85285EF20BB
:10095000405019C1EF2020707C40FD177CC07C40C6
:100960006354F0001C48FDF323223405EF203008C7
:10097000EF10700F31F1593C054B81B73C41E38FCB
:1009800007E27370043001A07370043001A030409E
:1009900021E61C4085C71C5C585085071CDC39FBD0
:1009A000EF20F0040545B640264496440649F25926
:1009B000625AD25A425BB25B616182804840EF204A
:1009C00020781C5C58502322040085071CDCE313AC
:1009D00007F279D5253CE9B74844A685EF30700C7D
:1009E0003C4058441440B307F0403E9758C4637CE1
:1009F000D7025840BA975CC409475C506306E902C5
:100A0000185C050718DCC9DFF5B54844A685EF304A
:100A100050093C4058441440B307F0403E9758C436
:100A2000E37CD7FCF9B75C50185C79DB185C7D1768
:100A300018DC185C050718DCA5D76DBD2285953E2E
:100A4000EF107002014585B7EF20607A0145A1BF24
:100A5000411126C2AA841305400522C406C6EF3000
:100A6000006C2A8415CD232C0502FD577CC1054757
:100A7000410558DC3CC42322040023200400232425
:100A80000400232604002320040423089404413492
:100A900013054402AD3C8146014681452285013360
:100AA0002285B24022449244410182800DC5411109
:100AB00022C426C206C64AC0032945002A84EF2064
:100AC000405B8144630CA900B24022442685024960
:100AD0009244410182807370043001A05C448544DB
:100AE000FD175CC4F5F381460146814522854539F1
:100AF000E1BF397106DE22DC26DA4AD84ED652D45E
:100B000032C635CD8149DDC13689AE842A84130AC7
:100B100005012DA0EF20A06DEF20206B6C002808B0
:100B2000EF20604831E1EF20406A185C5C5C6305AF
:100B3000F702EF20C06BEF20806B8549EF20E06863
:100B4000185C5C5C6360F704B24799CFE39409FCDE
:100B50002808EF2020437DBFEF206069B245528511
:100B6000EF20E0106530C1BFEF206068F2506254A2
:100B7000D2544259B259225A014521618280737080
:100B8000043001A0304015EE1C4095C71C5C585045
:100B900085071CDC39E7EF208065F2506254D2549F
:100BA0004259B259225A0545216182803C41A9DF50
:100BB0007370043001A04840EF20805823220400C5
:100BC000F1B7631909020844A685EF30806D1C4413
:100BD00034405840B6971CC4E3EAE7FA1C401CC4F2
:100BE00075B713054402EF20C0268547E315F5FAD3
:100BF000313855B74844A685EF30A06A3C40584488
:100C00001440B307F0403E9758C46375D70058406E
:100C1000BA975CC48947E31BF9F61C5CA5DB1C5C36
:100C2000FD171CDCA5B7397106DE22DC26DA4AD8AE
:100C30004ED652D432C66301050E81446388050C3A
:100C4000B6892E892A84130A450231A0EF20205A42
:100C5000EF20E0598544EF2040571C5CBDE3B247CC
:100C600095CF8DC8EF20A058EF2020566C002808A3
:100C7000EF20603305E5EF2040551C5CE1FBEF20E1
:100C800000571C409DC7B2455285EF10507EEFF0D3
:100C9000EFF77DBF2808EF20E02EE9B7EF202055C1
:100CA000F2506254D2544259B259225A014521613C
:100CB0008280EF2080514840EF20603EEF2020539B
:100CC000D9B73040444409CE5840B387C4005CC40F
:100CD00063E4E7001C405CC44C444A85EF30605C30
:100CE000639F09021C5C1840FD171CDC01E7EF2024
:100CF000805448C01C489DC713050401EF206015AF
:100D000085476311F502EFF06FF029A83C41E389B4
:100D100007F27370043001A07370043001A05C50BE
:100D200044C481EFEF20A04CF2506254D254425997
:100D3000B259225A05452161828013054402EF20F1
:100D400040116DD1C9B725C1B1C9011122CC26CA44
:100D50004AC852C406CE4EC68947B68432892E8A06
:100D60002A846399F600585D85476301F70673701E
:100D7000043001A0EFF06FF5185C5C5CAA89636732
:100D8000F70281444E85EFF0EFF3F240624426858E
:100D90004249D244B249224A056182803C41D5D7BA
:100DA0007370043001A07370043001A0304049E238
:100DB0001C40DDCB1C5C7D5785071CDC3C446388F4
:100DC000E7083C44854485073CC46DBFEFF0EFEF76
:100DD000185C5C5CAA89636DF702304071DA4844A4
:100DE000D285EF30004C3C4058441440B307F040EB
:100DF0003E9758C46375D7005840BA975CC489477A
:100E0000E39AF4FA1C5CDDD71C5CFD171CDC5DB7B3
:100E1000304059DE4844D285EF30A0483C40584429
:100E20001440B307F0403E9758C4E367D7FCD9BFDE
:100E3000DDF40844D285EF30C0461C4434405840AD
:100E4000B6971CC4E3E8E7F61C401CC4A5B75C5089
:100E500085448DDB13054402EF10B07F05D5E30315
:100E600009F22320990039BF4840EF20602D23224A
:100E7000040089B731CD3C4181C77370043001A0B3
:100E80001C41B1CB011122CC26CA2A844AC84EC6C5
:100E900006CE2E89EFF06FE3185C5C5CAA89814472
:100EA000637DF7001C5C7D5785071CDC3C4463892F
:100EB000E7023C44854485073CC44E85EFF08FE053
:100EC000F240624426854249D244B249056182809B
:100ED0007370043001A05C41D5D77370043001A059
:100EE0005C5099E38544D1BF13054402EF1070763E
:100EF00075D9E30909FE85472320F900E5B7397163
:100F000006DE22DC26DA4AD84ED652D456D232C673
:100F10006302051C638A051AB68AAE892A84EF200B
:100F2000001611E5B24781C77370043001A0EF20AD
:100F3000C0291C5C63920714B247638E070A280815
:100F4000EF204004FD5413094402130A0401EF206A
:100F5000002AEF10400CEF2040277C40639497005C
:100F6000232204043C446394970023240404EF20C8
:100F700000286C002808EF20000363130518EF20F9
:100F8000C0241C5CADCFEF208026EF2000243C4421
:100F9000634FF00039A84A85EF10B06B19C1EF20FC
:100FA000800B3C44FD173CC43C446354F0005C504F
:100FB000FDF324C4EF20A023EF2020217C40634FC9
:100FC000F00039A85285EF10D06819C1EF20A008B1
:100FD0007C40FD177CC07C406354F0001C48FDF34E
:100FE00064C0EF20C020EF100028EF20001E1C5C22
:100FF000C1E7B247A9FFEF20801F014555A0EF20B0
:10100000001F1C40DDC7B2454A85EF105046EF2057
:10101000C01B3C44634FF00039A84A85EF10706351
:1010200019C1EF2040033C44FD173CC43C446354C9
:10103000F0005C50FDF324C4EF20601BEF20E018AB
:101040007C40634FF00039A85285EF10906019C1C1
:10105000EF2060007C40FD177CC07C406354F000B2
:101060001C48FDF364C0EF208018EF10C01F31C989
:10107000EF20A0151C5CB5DFCE8522854444EFF03F
:101080006FD1639C0A041C5C1840FD171CDC01E74F
:10109000EF20601A48C01C48A1EFEF20401505451D
:1010A000F2506254D2544259B259225A925A216192
:1010B0008280EF2080114840EF10707EEF202013D7
:1010C00099B7EFF0AFB46DB73C41E38707E47370B5
:1010D000043001A07370043001A05C5044C4D5DF1B
:1010E00013054402EF10F0564DD9EFF02FB275B74B
:1010F00013050401EF10F0558547E310F5FAF5B735
:101100002285EFF00FCBEF100016014551BF1DC92E
:10111000411122C44AC006C626C244412E892A84EF
:10112000EF1030756383A40281464A86814522858B
:10113000F93385476300F502B240224492440249E4
:10114000410182807370043001A05C44054585072D
:101150005CC4DDB75C4485075CC4F9BF15CDADC97F
:10116000011122CC26CA4AC84EC652C42A8406CED1
:101170003289AE89EFF06FB51C5C2A8A814485E321
:101180005285EFF02FB4F240624426854249D244A2
:10119000B249224A056182807370043001A0304058
:1011A00001CE4C445C40B2954CC463E4F5000C4065
:1011B0004CC44E85EF30E00E1C5C7D57FD171CDCE7
:1011C0007C40638CE7007C40854485077CC04DBF34
:1011D0003C41D9D77370043001A01C4899E3854481
:1011E00045B713050401EF10D04675D9E30909FE90
:1011F00085472320F900E5B721C93C41A1CDA1CB0A
:10120000011122CC26CA4AC852C42A8406CE4EC630
:101210002E8AEFF08FAB1C5C2A89814491CB832905
:10122000C400D2852285EFF0EFB685442326340131
:101230004A85EFF02FA9F240624426854249D24404
:10124000B249224A056182807370043001A0737034
:10125000043001A0EDDF7370043001A001E573706C
:10126000043001A0411122C42A8406C6EF10F07593
:10127000005CEF10D077B240228522444101828089
:1012800001E57370043001A0411106C622C42A840E
:10129000EF10B0731C5C405C1D8CEF105075228504
:1012A000B24022444101828019C1085D828073707E
:1012B000043001A01DCD978703009387A750D84322
:1012C000630CE502D847630CE504D84B6307E504DB
:1012D000D84F6302E504D853630DE502D85763087D
:1012E000E502D85B6303E502D85F630EE5006F207B
:1012F00030757370043001A001470E07BA9723A020
:1013000007006F20F0731D47CDBF1947FDB7154784
:10131000EDB71147DDB70D47CDB70947F9BF054711
:10132000E9BF684582806CC58280034505058280DF
:1013300009C5085D1335150082807370043001A063
:1013400019C51C5D485D1D8D1335150082807370B5
:10135000043001A0978703009387C746984305C3CD
:10136000984705C7984B05C7984F05C7985305C7B9
:10137000985705C7985B15C7985F15C382800147CA
:101380000E07BA978CC3C8C382800547D5BF0947EB
:10139000C5BF0D47F5B71147E5B71547D5B71D4789
:1013A000C5B71947F1BF978703009387A741D84373
:1013B0006308E502D847630BE502D84B630AE502F0
:1013C000D84F6309E502D8536308E502D85763078D
:1013D000E502D85B6308E502D85F6303A702828059
:1013E00001470E07BA9723A0070082800547D5BFA3
:1013F0000947C5BF0D47F5B71147E5B71547D5B73D
:101400001D47C5B71947F1BF411122C426C24AC0C2
:101410002A8406C6AE843289EF10305B7840FD57CF
:101420006314F700232204043844FD576314F700C3
:1014300023240404EF10B05B1C5C99E74A86A68560
:1014400013054402EF10B015EF1030583C44635BB5
:10145000F0025C5085CB9304440209A83C44FD177C
:101460003CC43C446350F0025C5089CF2685EF10A9
:10147000501E6DD5EF10303E3C44FD173CC43C443B
:10148000E344F0FEFD573CC4EF107056EF10F053EC
:101490007C40635BF0021C4885CB9304040109A8DF
:1014A0007C40FD177CC07C406350F0021C4889CF13
:1014B0002685EF10101A6DD5EF10F0397C40FD171E
:1014C0007CC07C40E344F0FEFD577CC02244B24027
:1014D0009244024941016F10905197F701009387A0
:1014E000E709944317F70100130707081843C8C218
:1014F000636EE502411122C406C617F70100130707
:10150000A7072A8408438C439105EFF06F8397F770
:1015100001009387A7039C436376F40097F70100CB
:1015200023A68702B24022444101828017F70100BE
:101530001307470408438C4391056FF06F8097F7BA
:1015400001009387A703984394437C43FD177CC312
:10155000FC4299E37360043082801DC179714ECEE4
:1015600056CA06D6BE8A22D426D24AD052CC5AC8EF
:101570005EC69147BA8963F8E7007370043001A032
:101580007370043001A02A8BAE843289B68B428AF4
:101590006308082213050006EF2070382A84630CC4
:1015A00005200A09232845034A869305500A5285D7
:1015B000EF20305D03C704001C587119230AE402B0
:1015C00003C704003E991379C9FF79C783C7140084
:1015D000A30AF40283C71400E1C383C72400230BCA
:1015E000F40283C72400CDCB83C73400A30BF402DD
:1015F00083C73400D5C383C74400230CF40283C7D8
:101600004400D9CB83C75400A30CF40283C7540011
:10161000C1C783C76400230DF40283C76400ADCF44
:1016200083C77400A30DF40283C77400B5C783C7D2
:101630008400230EF40283C78400B9CF83C79400CB
:10164000A30EF40283C79400A1CB83C7A400230F89
:10165000F40283C7A400A9C383C7B400A30FF40294
:1016600083C7B40095CB83C7C4002300F40483C7A9
:10167000C4009DC383C7D400A300F40483C7D4006F
:1016800081CF83C7E4002301F40483C7E40089C742
:1016900083C7F400A301F404130A44005285A30194
:1016A00004042326340323283405232A0404EFE00A
:1016B0005FE713058401EFE0DFE69547B387374125
:1016C000232C040400C81CCC40D023220404232E65
:1016D00004045E86DA854A85EFE0DFDF08C06384B4
:1016E0000A0023A08A007370043017F9010013095F
:1016F00029E78327090097F40100938424E891C720
:1017000098409C407C4385077CC317F70100130772
:10171000E7E51C43850797F6010023A9F6E49C4002
:10172000CDCB8327090089EB9C40DC5763E6F900A9
:1017300097F7010023A487E497F70100938747E117
:101740009C4317F701001307E7E148541843850746
:1017500097F6010023AEF6DE3CC46376A70097F748
:10176000010023A1A7E0D145EF40106097F70100E9
:10177000938707F13E95D285EFE01FDB83270900B1
:1017800089C79C40FC436395070E832709000544E5
:1017900099C79C40DC5763F43701EFE03FC72285CF
:1017A000B250225492540259F249624AD24A424BF0
:1017B000B24B456182805285EF2090287D54C5B799
:1017C00013152600EF20B0152A8AE31505DC7D5499
:1017D000F9B797F7010023A387DA18438547E31D7C
:1017E000F7F417F501001305A5E9EFE05FD217F54F
:1017F0000100130525EAEFE09FD117F5010013055D
:10180000A5EAEFE0DFD017F50100130525EBEFE0C7
:101810001FD017F501001305A5EBEFE05FCF17FB15
:101820000100130B2BEC5A85EFE07FCE97FA0100F5
:10183000938A8AEC5685EFE09FCD17F501001305DA
:10184000E5ECEFE0DFCC17F50100130565EDEFE007
:101850001FCC17F501001305E5EDEFE05FCB97F71F
:10186000010023AB67D197F7010023A557D1E9B554
:10187000984094407C43FD177CC3FC42E39707F0FB
:101880007360043019B7411122C406C626C24AC08B
:101890002A847370043097F40100938464CC9C40D4
:1018A000F9E311E497F70100938747CD80431309CB
:1018B00044004A85EFE0DFCB1C5489C7130584013F
:1018C000EFE01FCBCA8517F50100130565E5EFE0D2
:1018D000BFC597F701009387A7C9984397F7010001
:1018E000938707C79C43050797F6010023A2E6C824
:1018F0009840850797F6010023ACF6C401CB97F713
:1019000001009387A7C79843784349EF9C40B1C72C
:1019100097F70100938787C69843630F8708737012
:101920000430984039EB17F701001307E7C414435C
:101930009442A5E27D5797F6010023A9E6C098409E
:1019400009CF9843784311CB984394437C43FD17C8
:101950007CC3FC4299E373600430B2402244924459
:1019600002494101828097F70100938727C198437C
:101970009C437C4385077CC32DB794439843F8422E
:101980000507F8C217F70100130707BF1443944275
:10199000D5D2184358475847584397F6010023A714
:1019A000E6BA71BF984394437C43FD177CC3FC4265
:1019B000B1FF7360043099BF97F701009387C7B8F0
:1019C0009C4381C77370043001A02244B24092440A
:1019D000024941016FE09FA341C517F701001307BA
:1019E000E7B914438147638BA606411106C622C49A
:1019F00026C27370043097F60100938666B69C4247
:101A000091C710431C437C4285077CC29C42AA8438
:101A1000404981C71C43FC43B9E797F7010093870E
:101A2000A7B59C43638A870497F70100938787B41F
:101A30009C436383870497F701009387A7CF6308CC
:101A4000F40297F701009387A7CD6300F40285475E
:101A5000B240224492443E85410182803E8582808C
:101A60007370043001A0E13C4DBF9147D5B79C5441
:101A700093B717008907E9BF8947D9BF737004304E
:101A800097F701009387C7AD984309EF15C59C43AD
:101A9000485581CB97F70100938747AE9843784329
:101AA00015E3828017F70100130747AD144318436D
:101AB000F8420507F8C261FD17F70100130707ACEC
:101AC0000843F1B7984394437C43FD177CC3FC4221
:101AD000E9FB736004308280411122C42A8406C667
:101AE000EFE0BF9E11E497F70100938727A9804399
:101AF0004054EFE03F9DB240228522444101828064
:101B0000914763F5B7007370043001A0011122CC36
:101B100006CE26CA4AC84EC652C42A847370043000
:101B200017F901001309C9A383270900CDEF71C478
:101B30003C486388F50817F70100130727A463FCE6
:101B4000B7001443638B860C18434457B3B4950015
:101B500093C4140029A00443818C93B414005854F6
:101B60006383E70A1C4C2CC863C607009547B385FE
:101B7000B7400CCC93172700BA97584897F9010043
:101B8000938909B08A07CE97631AF702130A4400B3
:101B90005285EFE0FF9D97F701009387A79C48547B
:101BA0009C4363F6A70097F7010023ADA79AD145A0
:101BB000EF40901BD2854E95EFE01F9799C0EFE064
:101BC000FF848327090081CB97F701009387079B48
:101BD0009C43FC439DEBF2406244D2444249B249EB
:101BE000224A0561828097F70100938727999843DD
:101BF0009C437C4385077CC305FC97F701009387D2
:101C0000E797804335B74CD4B1BF6244F240D24429
:101C10004249B249224A05611DB2814489B725C1B2
:101C2000011126CA97F40100938444959C4006CE86
:101C300022CC4AC84EC6638DA7027370043017F9D0
:101C400001001309E9918327090091C798409C403E
:101C50007C4385077CC3584997F70100938787AD7C
:101C60006302F7028327090081C79C40FC43A5EB70
:101C7000F2406244D2444249B249056182807370A5
:101C8000043001A01C5517F70100130727A8E38BA8
:101C9000E7FCE9FB930945002A844E85EFE05F8D60
:101CA00097F701009387078C48549C4363F6A7007D
:101CB00097F7010023A8A78AD145EF40F00A97F7CC
:101CC00001009387E79B3E95CE85EFE0FF859C4022
:101CD0005854DC57E368F7F8EFE04FF361B762441C
:101CE000F240D2444249B249056191B815CD011183
:101CF00022CC26CA4EC62A8406CE4AC8EFE0EFFCA4
:101D0000584897F701009387E7A2AA8981446300A6
:101D1000F7024E85EFE00FFBF24062442685424910
:101D2000D244B249056182807370043001A01C5412
:101D300017F501001305859DE38DA7FCF9FB97F7C7
:101D40000100938767809C43A9EB97F70100938775
:101D5000E7829C43445413094400DC574A85B3B4DA
:101D6000F400EFE0FF8097E701009387A77F4854D6
:101D70009C4393C4140063F6A70097E7010023A3D4
:101D8000A77ED145EF40407E97F701009387478FAC
:101D9000CA853E95EFE04FF9ADBF93058401EFE0B2
:101DA000AFF885BF0111056506CE22CC26CA4AC808
:101DB0004EC652C456C2EF208036630E051CAA845C
:101DC00013050006EF20A0352A84630A051E056668
:101DD0009305500A04D92685EF20A05A0458856738
:101DE000F117BE94B7474C45938797449309440035
:101DF0005CD84E85230C0402A301040423260402AC
:101E000023280404232A0404EFE0AFF1130584011E
:101E1000EFE02FF19547232C0404F19800C81CCC67
:101E200040D023220404232E040401469715000009
:101E30009385E5B12685EFE0EFE908C073700430C3
:101E400017E901001309C9718327090097E401000C
:101E50009384C47291C798409C407C4385077CC39F
:101E600017E70100130787701C43850797E60100F9
:101E700023AEF66E9C40C9C38327090081EB9C40CA
:101E8000DC5789E797E7010023AA876E97E70100EF
:101E90009387076C9C4397E601009386A66C585481
:101EA0009442850717E601002324F66A3CC463F6D2
:101EB000E60097E7010023A7E76A93172700BA9780
:101EC0008A0717E501001305A57B3E95CE85EFE057
:101ED000AFE58327090081C79C40FC43F1E78327D6
:101EE000090091C39C40EF10F04985476304F50E4B
:101EF0005DE17370043001A097E7010023A08768BB
:101F000018438547E314F7F817E5010013054577F3
:101F1000EFE0EFDF17E501001305C577EFE02FDFF6
:101F200017E5010013054578EFE06FDE17E50100C6
:101F30001305C578EFE0AFDD17E50100130545791E
:101F4000EFE0EFDC97EA0100938ACA795685EFE06B
:101F50000FDC17EA0100130A2A7A5285EFE02FDB23
:101F600017E501001305857AEFE06FDA17E5010048
:101F70001305057BEFE0AFD917E501001305857B5D
:101F8000EFE0EFD897E7010023A8575F97E701003C
:101F900023A2475FE5BDF2406244D2444249B249C0
:101FA000224A924A05618280984094407C43FD1702
:101FB0007CC3FC42E39507F2736004300DB76244C2
:101FC000F2404249B249224A924A2685D2440561EA
:101FD0006F20002773700430FD5717E70100232797
:101FE000F756624497E7010023ACA756F240D2446B
:101FF0004249B249224A924A97E7010023A607566E
:1020000005616FE00FAA7370043097E7010023A900
:1020100007546FE04FB717E701001307E7521C435F
:1020200085071CC382807370043097E70100938793
:102030002753984305E317E701001307E7520843C6
:102040009C4381CB97E7010093874753984378439C
:1020500001EF828017E7010013074752144318432A
:10206000F8420507F8C2C1BF984394437C43FD176B
:102070007CC3FC42F9FF736004308280411106C6C4
:1020800022C4EFE08FC497E701009387E74D8043B8
:10209000EFE04FC3B240228522444101828097E79E
:1020A00001009387A74C88438280797106D622D499
:1020B00026D24AD04ECE52CC56CA5AC85EC697E7F0
:1020C0000100938767489C43B1EF17E701001307AE
:1020D000A7491C43850797E6010023A7F648832AF2
:1020E0000700638F0A0697E70100938727469C4302
:1020F000814463F1FA0897E901009389695817EA66
:102100000100130AAA4783270A008546D857931768
:102110002700BA978A07BE9983A7090063FFF600D4
:10212000854421A897E70100938747439C43814456
:10213000850717E701002323F74297E701009387FC
:10214000A7419C4391C38544B2502254268502592D
:102150009254F249624AD24A424BB24B4561828064
:1021600017E40100130444411C409C43DDC3737019
:10217000043001A017E401001304044097E90100B2
:102180009389095017EA0100130A4A3F17EB01002F
:10219000130B4B3D1C409C43B5C31C40DC4703A9BB
:1021A000C70083274900930B49005E8563EEFA045C
:1021B000EFE00FBC832789021305890199C3EFE083
:1021C0002FBB8327C90203270B00DE851395270049
:1021D0003E950A054E956376F70017E70100232325
:1021E000F738EFE06FB483270A000327C902DC57F2
:1021F000E362F7FA1C4085449C43C5F3FD5717E79B
:1022000001002325F73401B717E701002320F73435
:10221000DDBD17E701001307E7351C40184397E6BB
:10222000010023ABE63417E701002325F73497E7D5
:102230000100938727329C43850717E70100232B72
:10224000F7301C409C4399E7FD5717E70100232F07
:10225000F72E51BD1C40DC47DC47DC4317E701008B
:102260002326F72E49B597E701009387E72D98437A
:1022700001E77370043001A0011106CE22CC26CAFA
:102280004AC84EC652C456C25AC07370043097E44E
:1022900001009384E42C984061EB98437D1797E606
:1022A000010023A3E62A9C43D9EB97E7010093871B
:1022B000E72B9C43C9C797EA0100938A6A3C17EA57
:1022C0000100130A2A2A17E901001309292B85495D
:1022D00019A83385EA00EFE02FA583270900585499
:1022E000DC576379F70483A7CA08C1CF83A78A099B
:1022F000C04713058401EFE0AFA7130B44005A85D4
:10230000EFE00FA75C5483260A00DA8513952700B7
:102310003E950A052A875695E3FDF6FA17E7010070
:102320002322F724EFE04FA0832709005854DC57FD
:10233000E36BF7FA97E7010023A037236DB7014459
:102340009C4081CB97E70100938747239C43FC4344
:1023500095E72285F2406244D2444249B249224A7A
:10236000924A024B0561828017E70100130707219B
:1023700014431843F8420507F8C205B7EFF02F9C45
:10238000C9BF17E401001304641D1C4095C31C4021
:10239000054999CF193B09C597E7010023AE271BD3
:1023A0001C40FD1717E70100232AF71A1C40FDF314
:1023B00097E701009387471A98438547E311F7F899
:1023C000EFE0CF840544ADBF11CD81E573700430DB
:1023D00001A017E70100130727171C4399C7737063
:1023E000043001A07370043001A0411122C406C65C
:1023F00014431841850617E601002327D61497E6F3
:1024000001009386661694423304B70000C163F757
:10241000E602637FE40063FD860097E7010093878F
:10242000E71588431105EFE0AF942285EFF0EF8ABE
:102430001D3D01C9B240224441018280E36FE4FCAA
:10244000D9BF2244B24041016FD05FFC11C917E7E8
:1024500001001307670F1C4391C77370043001A07C
:102460006FD0DFFA411106C622C41843AA870507B8
:1024700097E6010023AAE60C97E601009386061072
:1024800017E701001307470E184388423304F7008B
:102490001105EFE0EF8D2285EFF02F84E93311E590
:1024A0002244B24041016FD07FF6B2402244410144
:1024B0008280411122C406C697E701009387C708AE
:1024C0009C430144850717E70100232FF70697E790
:1024D00001009387A7099C4363E3F50C17EE010005
:1024E000130E8E1F97E201009382C2180144014728
:1024F000854F1303500A21A0311E6387C20D832725
:102500008EFFBA85F5DB8327CEFFDC43232EFEFE4C
:102510006382C71B03AFC700DC432A97814E232E7B
:10252000FEFE6385C70783A8C7009387480323205F
:1025300017015CC383A788042326F7011CC783A760
:10254000C8021CCB83A70805232C07005CCB03A87B
:10255000080383470800639A6704C287850783C618
:102560000700B3850741E38B66FE8981C205C181FF
:10257000231EB700850E1307070263001F0583277C
:10258000CEFFDC43232EFEFEE39FC7F983274E00D8
:10259000232EFEFE49BF1A9419C223200600E13102
:1025A0002285B2402244410182808145231EB7002A
:1025B000850E13070702E3141FFD769413175400CA
:1025C000311EBA85E39DC2F397E701009387C7FAEE
:1025D00003AE070083270E00FDE397E70100938712
:1025E00067F903AE070083270E006398071617EEFE
:1025F0000100130EEE0883270E0A639D071E832732
:102600004E0BD9DB83278E0B97EE0100938E0E13B2
:10261000DC4317E701002321F7126381D73383AF2F
:10262000C700DC433307B500014397E6010023A54B
:10263000F6100D4F89429308500A6386D707C847A2
:102640009307450308C35CC33C452326E7011CC729
:102650005C551CCB1C5599C3232657003C49232CA1
:1026600007005CCB03280503834708006395172BFD
:10267000C287850783C60700B3850741E38B16FF32
:102680008981C205C181231EB70005031307070214
:10269000E383AFF083278E0BDC4397E6010023AD85
:1026A000F608E39ED7F983270E0C97E6010023A5D1
:1026B000F60871B783274E00232EFEFEA1BD8327A7
:1026C0004E00130F8E00D4432322DE00638CE625D8
:1026D000B307E500D84283A2C600814E2322EE0054
:1026E000894F1303500A6305EF068328C700138739
:1026F000480323A01701D8C303A7880423A6F70122
:1027000098C703A7C80298CB03A7080523AC070006
:10271000D8CB03A80803034708006318671C428747
:10272000050783460700B3050741E38B66FE8981F1
:10273000C205C181239EB700850E93870702638E71
:10274000121B83264E00D8422322EE00E31FEFF82F
:102750000327CE002322EE0049BF83274E00130F2C
:102760008E00DC432322FE006389E71B83A2C7009F
:10277000DC43AA95814E2322FE00894F1303500AA1
:102780006305FF0683A8C7009387480323A01501AC
:10279000DCC183A7880423A6F5019CC583A7C802D2
:1027A0009CC983A7080523AC0500DCC903A808035E
:1027B0008347080063976710C287850783C60700B1
:1027C00033870741E38B66FE098342074183239EDB
:1027D000E500850E93850502638D120F83274E0059
:1027E000DC432322FE00E31FFFF88327CE002322D1
:1027F000FE0049BF83274E0A17EF0100130FCFF2E7
:10280000DC4317E70100232FF7F06382E71383A26D
:10281000C700DC43AA95814E17E701002324F7F097
:10282000914F1303500A6387E70783A8C700938774
:10283000480323A01501DCC183A7880423A6F50162
:102840009CC583A7C8029CC983A7080523AC0500C3
:10285000DCC903A808038347080063946704C287A0
:10286000850783C6070033870741E38B66FE09832C
:1028700042074183239EE500850E93850502638A06
:10288000120383274E0ADC4317E70100232CF7E8E5
:10289000E39DE7F98327CE0A17E701002324F7E831
:1028A00069B70147239EE500850E93850502E39AEB
:1028B00012FD83274E0B769493155400E38E07CCBC
:1028C00091B30147239EE500850E93850502E397AA
:1028D00012F117EE0100130EAEDA83270E0A76947A
:1028E00093155400E38D07D031B78145239EB7007F
:1028F000850E93870702E39612E597E70100938719
:1029000067C703AE070076949315540083270E0023
:10291000E38F07CC99B58145BDB38327CE00232231
:10292000FE00A9B58326CE002322DE0055B38327FF
:10293000CE0A17E701002327F7DED1BD83270E0C4F
:1029400017E70100232AF7DED9B9797126D24AD0D8
:102950004ECE52CC56CA5AC85EC606D622D497E985
:102960000100938969BE17E90100130969D117EACB
:102970000100130AEABE97EA0100938A2AC097EB86
:102980000100938BABBE97E40100938464BE054BBA
:1029900021A883A709000324090A850717E7010076
:1029A0002324F7BAC93011E89C40E5F783270900D2
:1029B000E37CFBFEEFD09FA5C5BF73700430832777
:1029C0000A00B9E38327C90AC04713054400EFD0C2
:1029D0003FBA83A70B00FD1717E701002328F7B8BC
:1029E0009C40FD1717E701002324F7B883270A004E
:1029F00089C783A70A00FC4385E30858EF105004F9
:102A00002285EF10F0034DB703A70A0083A70A0041
:102A10007C4385077CC37DB703A70A0083A60A0011
:102A20007C43FD177CC3FC42E9FB73600430F1B7C3
:102A300097E70100938747B19C43DDE7411106C644
:102A400022C426C297E7010023A807B017E70100B8
:102A50001307C7B21C43B7A6A5A59386565A9C5B1D
:102A60008C43639BD500D0436318B60094476395AD
:102A7000C600DC476388D70008430C4393854503B1
:102A8000EF20C07317E701001307C7AD144317E425
:102A900001001304E4BE11A81C43A9CF1C43FD1779
:102AA00097E6010023A0F6AC144393972600B6974F
:102AB0008A07A2979C43EDD3084393172500AA9752
:102AC0008A073307F4005443A107A297C44244C3C2
:102AD0006385F402DC44B240224417E70100232F4F
:102AE000F7A8924441018280854717E7010023251A
:102AF000F7A682807370043001A0C440D145EF3046
:102B0000B026229544C1F9B701114AC806CE22CC9D
:102B100026CA4EC62A897370043097E40100938454
:102B200024A49C4017E40100130444A5D9E76314CE
:102B3000090003290400930949004E85EFD05FA3E3
:102B40008327890289C713058901EFD07FA2CE852B
:102B500017E50100130505BEEFD01F9D9C4081C7FE
:102B60001C40FC43ADE31C40638B27079C409DCF7A
:102B7000737004309C40C1EB97E701009387C79FB7
:102B80009843184325EBFD5717E701002320F79CD6
:102B90009C4089CF1C40FC4391CB184014407C439F
:102BA000FD177CC3FC4299E373600430F240624439
:102BB000D2444249B2490561828018401C407C439E
:102BC00085077CC3ADB7184014407C43FD177CC318
:102BD000FC42D1FB736004301C40E39927F99C4010
:102BE000A1C397E70100938727969C43ADCB7370F1
:102BF000043001A09C43DC47DC47DC4317E70100BD
:102C00002326F79471B718401C407C4385077CC38A
:102C100097E7010093874796984318432DD7D9BF6C
:102C200097E701009387879417E70100130747A5EB
:102C30009C430327470B631DF700F240624497E76C
:102C4000010023AD0792D2444249B2490561828016
:102C50006244F240D2444249B2490561D1BB624468
:102C6000F240D2444249B24905616FD02FFA3DC9C2
:102C7000411126C297E40100938444904AC02E89F2
:102C80008C4006C622C4E105EFD09F8B8840110519
:102C9000EFD01F8EFD57630AF90497E70100938771
:102CA000A78C804398409C434A9440C3636CF404CF
:102CB00097E701009387478C88438C409105EFD0BC
:102CC0003F8897E70100938767889C436376F40009
:102CD00097E7010023AC8786B24022449244024920
:102CE000410182807370043001A08C402244B240C4
:102CF0009244024917E501001305C5A3910541015E
:102D00006FD09F8297E701009387C786884322444C
:102D10008C40B24092440249910541016FD05F82DC
:102D200011C997E70100938727829C4399E7737045
:102D3000043001A07370043001A0411126C297E451
:102D400001009384A4839840AE878C40B70600802E
:102D5000D58F06C622C41CCFE1053284EFD0CFFC4C
:102D600088401105EFD0DF80FD57630EF40097D740
:102D700001009387677F8843B240924422952244A2
:102D800041016FE08FF58C402244B240924417E538
:102D900001001305259A910541016FD0EFF825CD6B
:102DA000411126C297D401009384447D4AC02E89E4
:102DB0008C4006C622C4E1053284EFD0EFF688408D
:102DC0001105EFD0EFFA8547630AF40497D70100A5
:102DD00093878779804398409C434A9440C3636CAF
:102DE000F40497D701009387277988438C40910595
:102DF000EFD00FF597D70100938747759C43637613
:102E0000F40097D7010023A38774B2402244924470
:102E10000249410182807370043001A08C40224439
:102E2000B2409244024917E501001305A5909105AF
:102E300041016FD06FEF97D701009387A773884345
:102E400022448C40B24092440249910541016FD026
:102E50002FEF411106C622C426C25C45C04735CCBF
:102E6000930484012685EFD0AFF097D701009387B4
:102E7000A76D9C43B5E7930444002685EFD04FEF40
:102E800097D701009387076E58549C4363F6E70079
:102E900097D7010023A8E76C93172700BA978A07F2
:102EA00017D501001305C57DA6853E95EFD0CFE768
:102EB00097D701009387876C9C4358540145DC5792
:102EC00063F8E700854717D701002327F768054512
:102ED000B24022449244410182807370043001A0C8
:102EE000A68517E5010013056582EFD0EFE3C9B7AA
:102EF00097D70100938747659C4381E7737004303F
:102F000001A0411106C622C426C2B7070080404571
:102F1000CD8F1CC12DC4EFD0AFE5930444002685AE
:102F2000EFD00FE597D701009387C76358549C43B0
:102F300063F6E70097D7010023A6E76293172700FF
:102F4000BA978A0717D50100130585733E95A685A4
:102F5000EFD08FDD97D70100938747629C43585489
:102F60000145DC5763F8E700854717D701002325A3
:102F7000F75E0545B240224492444101828073705D
:102F8000043001A011CD97D701009387A75C984327
:102F900097D701009387475D9C4318C15CC182802D
:102FA0007370043001A055C1D1CD411106C622C4B1
:102FB0002A877370043097D801009388685A83A7D2
:102FC000080091CB97D701009387475B94439C43BC
:102FD000FC428507FCC217D301001303E3589C4150
:102FE00003260300FD560144638FD70217DE01005C
:102FF000130E4E5603250E000328070054436305A5
:10300000A80005446371D6023308D6400544637CAA
:10301000F80003250E00918F03260300B6979CC18C
:1030200008C350C3014483A7080081CB97D7010090
:103030009387C7549C43FC4381EF2285B2402244CE
:10304000410182807370043001A07370043001A0CC
:10305000EFE0EFCEDDB7854717D70100232EF74EFF
:10306000828019C1684582800145828011C16CC58A
:10307000828097D70100938767508843828097D7D3
:1030800001009387E74D9C43054589CB97D7010005
:103090009387874B8843133515000605828031CD11
:1030A000011126CA97D401009384444D9C4006CE5A
:1030B00022CC4AC84EC65855DC576379F7021C4DDE
:1030C00063C707009C40D4579547958F1CCD931735
:1030D0002700BA97584917D901001309695A8A0776
:1030E000CA97630DF7009C40DC575CD5F240624400
:1030F000D2444249B24905618280828093094500E9
:103100002A844E85EFD0CFC69C4017D70100130705
:1031100067451843DC575CD46376F70017D7010086
:103120002322F744139527003E9562440A05F24096
:10313000D244CE854A95B249424905616FD0CFBE8F
:1031400019CD411106C622C426C297D70100938724
:10315000E74280436307A4007370043001A0014577
:1031600082807C4881E77370043001A05454384851
:10317000FD177CC86383E60099C70145B24022442D
:10318000924441018280930444002685EFD04FBED3
:10319000284897D701009387E73C98439547898F44
:1031A00048D41CCC6376A70097D7010023ACA73A7C
:1031B000D145EF30603B97D701009387674C3E9530
:1031C000A685EFD06FB6054555BF7370043097D70D
:1031D00001009387E7389C4391CB97D701009387F1
:1031E000E73998439C437C4385077CC3828097D70B
:1031F00001009387E7369C438DC397D701009387DF
:10320000E7379843784311CB984394437C43FD17A9
:103210007CC3FC4299E373600430828097D701003D
:103220009387C7359043944398439547D456084EA7
:10323000958F1CCF828097D70100938727349843BE
:1032400009C79443F84A0507F8CA88438280797110
:103250004AD006D622D426D24ECE2A8973700430A4
:1032600097D401009384C42F9C4017D40100130409
:10327000E430BDE31C40BC4F89E71C400547F8CF54
:10328000D1E19C4081C71C40FC43F1EB73700430DA
:103290009C408DEF1C40A84F11C5630409021C40DF
:1032A00023AC07041C4023AE07049C4081C71C408C
:1032B000FC438DEBB250225492540259F2494561BD
:1032C000828018403C4FFD173CCFE9BF18401C409E
:1032D0007C4385077CC37DBF18401C407C43850729
:1032E0007CC349BF184014407C43FD177CC3FC429B
:1032F000F1F373600430B250225492540259F249EF
:103300004561828008402EC61105EFD06FA6B245F8
:10331000FD576380F50697D701009387E72483A9BB
:10332000070018409C43AE992322370163ECF9044F
:1033300097D701009387472488430C409105EFD02D
:103340002FA097D70100938767209C4363F6F9006D
:1033500097D7010023AC371FEFD04F8B1DB7184014
:1033600014407C43FD177CC3FC428DF37360043032
:1033700031BF0C4017D501001305C53B9105EFD0B7
:10338000AF9AD9BF97D701009387C71E88430C40D7
:103390009105EFD0EF9AC9B779714AD04ECE06D6D3
:1033A00022D426D252CC2E89B2897370043097D49D
:1033B00001009384E41A9C4017D401001304041CF8
:1033C000F9EF18408947784F630CF7001C4013450C
:1033D000F5FFB84F798DA8CF1C400547F8CFADE673
:1033E0009C4081C71C40FC43F5E3737004309C4053
:1033F000B1E7638609001C40BC4F23A0F9001840C8
:1034000085470145784F630BF7001C401349F9FFCE
:103410000545B84F3379E90023AC27051C4023AE9E
:1034200007049C4081C71C40FC43C1E3B2502254B6
:1034300092540259F249624A4561828018401C4008
:103440007C4385077CC375B7084036C61105EFD0AD
:103450002F92B246FD576385F60897D701009387F0
:10346000A71003AA070018409C43369A232247015D
:103470006363FA0897D701009387071088430C40CD
:103480009105EFD0EF8B97D701009387270C9C43D2
:103490006370FA0697D7010023AA470B91A818403A
:1034A0001C407C4385077CC329BF184014407C43E3
:1034B000FD177CC3FC42BDFB73600430B250225444
:1034C00092540259F249624A456182801840144080
:1034D0007C43FD177CC3FC4289FB7360043031B729
:1034E0000C4017D501001305E5249105EFD0CF83DB
:1034F000EFC0DFF1F5B597D701009387A7078843A1
:103500000C409105EFD0CF83E5B751C1411106C6FC
:1035100022C426C24AC07370043097D40100938439
:1035200024049C40B9EB99C23C4D9CC2B2878946A9
:10353000704D74CD2E872A846386D70663FCF6040B
:103540008D456387B70091456395B7006300D60C3E
:1035500038CC8547630FF60405449C4081CB97D750
:1035600001009387A7019C43FC43A9E32285B24055
:103570002244924402494101828097D701009387F7
:10358000E7FF98439C437C4385077CC369BF737006
:10359000043001A08546E39ED7FA3C4D33E7B700DF
:1035A00038CD45BF3C4D85073CCD65B7EFD03FF9E1
:1035B00075BF130944004A85EFC09FFB97D70100F0
:1035C000938747FA48549C4363F6A70097D70100B6
:1035D00023AAA7F8D145EF20307997D70100938728
:1035E000270A3E95CA85EFC03FF41C5481C773700B
:1035F000043001A097D70100938747F89C435854A3
:10360000DC57E3FBE7F4EFC07FE0B9B70144B1B7A3
:1036100039CD011122CC26CA4AC84EC652C456C260
:1036200006CEBA89368AB2842E892A84EFC0FFE991
:10363000AA8A63050A003C4C2320FA00784C89478B
:103640007CCC6389F40263F4970C8D466387D400C5
:1036500091466396D400630AF70A232C2405854714
:10366000631EF7061C5499CB7370043001A073706D
:10367000043001A03C4C85073CCCD5B797D701005E
:10368000938787EC9C43ADEB930444002685EFC001
:103690003FEE97D701009387E7EC48549C4363F6CD
:1036A000A70097D7010023AFA7EAD145EF20D06B41
:1036B00097D701009387C7FCA6853E95EFC0DFE64C
:1036C00097D70100938787EB9C435854DC5763F7E7
:1036D000E70063850900854723A0F9000544568566
:1036E000EFC05FDE2285F2406244D2444249B249D3
:1036F000224A924A056182809305840117D5010010
:103700001305C500EFC05FE265BF0144C9BF85472F
:10371000E397F4F43C4C33E92701232C240581B7CB
:103720004DC1011122CC26CA2A844EC606CE4AC8F3
:10373000AE84EFC09FD98947744C7CCC3C4C054784
:10374000AA8985073CCC6395E6061C5481C7737033
:10375000043001A097D70100938707DF9C43ADE7B2
:10376000130944004A85EFC0BFE097D70100938753
:1037700067DF48549C4363F6A70097D7010023A353
:10378000A7DED145EF20505E97D70100938747EF22
:10379000CA853E95EFC05FD997D70100938707DEB2
:1037A0009C435854DC5763F5E70099C085479CC09B
:1037B0006244F240D24442494E85B24905616FC02D
:1037C0007FD07370043001A09305840117D50100E8
:1037D0001305C5F3EFC05FD5C1B7AA8729C57370BC
:1037E000043017D701001307A7D714439DE2F04F09
:1037F000894601456315D60023AE070405451C43E1
:1038000081CB97D70100938767D79843784315E317
:10381000828097D60100938666D690429442744285
:10382000850674C2E9B797D70100938727D59C43D3
:103830007DB7984394437C43FD177CC3FC42E9FB6E
:103840007360043082805D71A6C2CAC052DC56DA51
:103850005AD85ED686C6A2C44EDE62D466D26AD07C
:1038600017D90100130989D217DB0100130B4BD1C3
:1038700097D40100938404D197DA0100938ACAD0C7
:10388000054AA54B83270900984363010712DC47CB
:1038900083A90700EFE02FF8EFE0EFF883270B0094
:1038A0002A8C6362F50A97D7010023ABA7CC0146A7
:1038B0006370351B8840B3858941EFD0FFB4EFE0DA
:1038C0009F9A630105128840814601462C00EFD083
:1038D0000FE34DD9A247E3C807FEC24983A74901B8
:1038E00089C713854900EFC0BFC8EFE0CFF3832736
:1038F0000B002A8C636DF508A24717D7010023211E
:1039000087C9E3E2FBFCB317FA0013F70721631A38
:10391000071613F7770C6318071E93F70702C5D72E
:103920004E85EF00F01145B7DC47C04783AC070078
:10393000930944004E85EFC0BFC35C502285829737
:103940005C4C6384470B83270900984371FF03A7EE
:103950000A0097D6010023A586C397D6010023A5A8
:10396000F6C297D7010023A3E7C2EFE0DF8FA1BF24
:10397000DC47C04703AD0700930C44006685EFC0E9
:103980003FBF5C50228582975C4C63864709832742
:103990000900984371FF03A70A0097D6010023A5E9
:1039A000F6BE97D7010023A3E7BEB9B7EFE0AFE6B5
:1039B000EFE06FE783270B002A8CE366F5F883A717
:1039C0000A00884081499043B385894117D7010097
:1039D000232887BB13361600EFD01FA3EFE0BF8864
:1039E000E31305EEEFC09FA2F9BD1C4CCE85E69710
:1039F00063E9FC049C4089CF02CA66CC22CEEFF07A
:103A00000FE88840814601464C08EFC05FD905FDAC
:103A10007370043001A01C4CE685EA97636CFD04CA
:103A20009C4089CF02CA6ACC22CEEFF04FE5884095
:103A3000814601464C08EFC09FD631F973700430BF
:103A400001A0032509005CC000C8EFC07FAFE5BD41
:103A5000EFE07F8183270900DC47C047930C4400D7
:103A60006685EFC0FFB05C4C638F47035C502285D6
:103A7000829791BD032509005CC000C8EFC05FAC10
:103A800039B7B24723ACF900A5CFE29723A2F900DA
:103A900023A8390193854900636FFC0403A50A003C
:103AA000EFC01FAA0DB51C4C00C83387F90058C0E1
:103AB000636DEC02330C3C416363FC029C4089CF94
:103AC00002CA4ECC22CEEFF08FDB88408146014601
:103AD0004C08EFC0DFCC59F97370043001A003A586
:103AE0000A00E685EFC0DFA551B703250900E6858A
:103AF000EFC01FA5A5BF03250900EFC07FA4E1B358
:103B00007370043001A0B24783A6890123A839014C
:103B10003387D70023A2E9006364EC04B307FC40B9
:103B200063EBD70483A749024E85829783A7C90117
:103B3000E39B47D983A68901B2479840B69711CF36
:103B400002CA3ECC4ECEEFF08FD38840814601466C
:103B50004C08EFC0DFC4E31805D67370043001A031
:103B60006374FC00E370F7FC0325090093854900AA
:103B7000EFC01F9D89BB03A50A0093854900EFC0D4
:103B80003F9C91B3411122C406C626C24AC017D435
:103B900001001304249FEFF04FE31C4095CBEFF09E
:103BA0000FE51C409DC38148014881470947814674
:103BB0001306004097D50100938545801705000046
:103BC0001305A5C8EFD07F9939E97370043001A0BF
:103BD00017D90100130949B74A85EFC05F9397D4FD
:103BE00001009384A4B72685EFC07F920146B145BA
:103BF000114597D7010023AB279997D7010023A53B
:103C00009798EFC0BFAC17D70100232DA79611CD11
:103C100097C501009385057AEFD0CFF349B7B2403D
:103C2000224492440249410182807370043001A011
:103C3000A5C9797156CAAA8A1305C00222D426D210
:103C40004AD04ECE52CC06D65AC85EC63A89B689FC
:103C5000328AAE84E9212A8405C9EFF00FD797D7BD
:103C60000100938727929C439DCFEFF04FD8130517
:103C700044002320540104CC232E44012320340388
:103C800023222403EFC0FF892285B250225492548C
:103C90000259F249624AD24A424BB24B4561828094
:103CA0007370043001A097DB0100938BEBA95E8554
:103CB000EFC0FF8517DB0100130B4BAA5A85EFC03D
:103CC0001F850146B145114597D7010023A0778D87
:103CD00097D7010023AA678BEFC05F9F17D701001A
:103CE0002322A78A01C997C501009385A56CEFD04F
:103CF0006FE6A5BF7370043001A039C5011122CC55
:103D000006CE26CA17D401001304C48783280400F2
:103D10002A88014563850802BA842EC2368732C4D8
:103D200042C6954663C5B602EFF06FB58947630B8F
:103D3000F5020840814601464C00EFC05FA6F24004
:103D40006244D244056182807370043001A04C004B
:103D500081463A864685EFC01FFFF2406244D24456
:103D6000056182800840814626864C00EFC03FA353
:103D7000F9B719C1084182807370043001A001E5D0
:103D80007370043001A0411106C622C42A84EFF0EA
:103D9000CFC348483334A000EFF06FC52285B2404E
:103DA00022444101828001E57370043001A0411179
:103DB00022C42A8406C6EFF04FC10050EFF02FC393
:103DC000B240228522444101828001E573700430B3
:103DD00001A0411122C426C22E84AA8406C6EFF097
:103DE000CFBE80D02244B240924441016FF02FC038
:103DF0004111714522C406C61D262A8411C52320FF
:103E000005001105EFC0AFF02285B2402244410108
:103E1000828001CDB70700FFED8F81C7737004303A
:103E200001A099E57370043001A07370043001A003
:103E3000011122CC4AC84EC652C456C206CE26CA6A
:103E4000BA893689B28A2E842A8AEFF04FA311E507
:103E5000638509007370043001A0EFE0CF9B8324D9
:103E60000A00B37794006316090295C763870A00B6
:103E70009347F4FFE58F2320FA00EFE0CFBEF24036
:103E8000624426854249D244B249224A924A056197
:103E90008280E30DF4FCE38209FEB3355001E205B4
:103EA00063050900B7070004DD8D4E86C18D13053B
:103EB0004A00EFE0FFE6EFE00FBB19E1EFC00FD5DE
:103EC000EFF0CFB593176500AA8963D80700B70450
:103ED0000001FD14B3F499005DB7EFF00FAF832933
:103EE0000A00B3773401631E090089CB63880A0096
:103EF0009347F4FFB3F737012320FA00EFF02FAF19
:103F0000F9B7E31DF4FEDDB701C9B70700FFED8F78
:103F100099C77370043001A07370043001A041117F
:103F200022C42A8406C626C24AC02E89EFF0EFA911
:103F300004409345F9FFB3F795001CC0EFF02FAB99
:103F4000B2402244268502499244410182804111B7
:103F500022C42A8406C6EFC04FD70040EFC08FD6D8
:103F6000B240228522444101828009C9370700FFFF
:103F7000B3F7E50099C77370043001A07370043083
:103F800001A06F20E06BB70700FFF18F81C773704E
:103F9000043001A001E67370043001A0011122CCAD
:103FA0004AC84EC652C406CE26CA3689AE892A8A67
:103FB0003284EFF0CF8C21E1630509007370043087
:103FC00001A0EFE04F8583240A00CE855285B3E43B
:103FD0009900613FB37794006307F40683240A00D5
:103FE000EFE06FA8F240624426854249D244B249CC
:103FF000224A05618280EFE00F8283240A00CE8589
:104000005285B3E434019537B3F78400638D87029A
:10401000E30609FCB70500054A86C18D13054A0071
:10402000EFE01FD0EFE02FA419E1EFC02FBEEFF0BB
:10403000EF9E93176500AA8463DF0700B7070001AE
:10404000FD17FD8C45B783270A001344F4FFE18F69
:104050002320FA0071B7EFF04F9783240A00B3775B
:104060009400639787009347F4FFE58F2320FA00BD
:10407000EFF0EF97E1B7411122C406C62A8426C2A9
:10408000EFD07FF95C4085C308489304C4006316F1
:10409000950015A0084863009502B7050002EFE0FF
:1040A0003FE55C40E5FB2285612A2244B240924410
:1040B00041016FE04F9B7370043001A009C93707BD
:1040C00000FFB3F7E50099C77370043001A0737067
:1040D000043001A06F20C05601C9B70700FFED8F63
:1040E00099C77370043001A07370043001A04111AE
:1040F00022C426C206C62A84AE84EFF00F8D184073
:1041000093C7F4FFF98F1CC02244B240924441018E
:104110006FF0EF8D19C1084D8280014582804111F9
:1041200022C406C62A84EFD01FEF97C701009387E9
:1041300027469C43A1EBE56717C701001307876378
:10414000F11797C6010023ABE64417C701002325EA
:10415000F74417C701002321F76297C7010093872F
:10416000674317C701002327F760854717C701007A
:104170002328074217C70100232E074017C7010055
:104180002328F74019E8EFE00F8EEF10A00201445A
:104190002285B24022444101828013058400937736
:1041A0003500C1EFE5671307F5FFE917E3EDE7FC1D
:1041B00097C601009386863E9C4229A0984311C76A
:1041C000BE86BA87D843E36BA7FE17C70100130763
:1041D000673CE38AE7FA984341461384870098C214
:1041E000D843B306A7406378D6023388A7002322BA
:1041F000D800C8C38325480097C601009386063AB5
:1042000011A0BA8698425043E36DB6FE2320E80021
:1042100023A00601D84397C701009387673B9C43BF
:10422000998F17C701002325F73AEFE0CF8331DCE0
:104230002285B240224441018280719911059DB7C7
:1042400029C9411122C406C62A84EFD0DFDC9305B8
:1042500084FF0326C4FF17C701001307273411A0EA
:104260003E871C43D443E3EDC6FE232CF4FE0CC36F
:1042700097C701009387C73598438327C4FF22441B
:10428000B240BA9717C701002324F73441016FD019
:104290009FFD828097C70100938787338843828080
:1042A00082803367B5000D8BAA871DE79308D6FF80
:1042B000AA982A87AE866371150303A80600110722
:1042C0009106232E07FFE36A17FF9347F5FFC69772
:1042D000F19B9107BE95AA972A9663F3C70A938626
:1042E000450013884700B3B6D70033B8050133E75C
:1042F000F50093C61600134818000D8BB3E60601AF
:1043000013371700758F330EF6409386170029CFA9
:104310001337AE0031EB13532E002E88BE860147B3
:10432000832808000507110823A016019106E369F8
:1043300067FE1377CEFFBA95BA976302EE0483C681
:104340000500138717002380D700637AC70283C64E
:10435000150013872700A380D7006372C70203C725
:1043600025002381E7008280B307F640AE978505DC
:1043700003C7F5FF8506238FE6FEE39AF5FE8280EC
:104380008280B367C5008D8BB308C500E9C3637134
:10439000150FB307A0408D8B13873700954693F513
:1043A000F50F130815003383A8407D166373D700FB
:1043B00015476363E60CD5CF2300B5000547638D31
:1043C000E700A300B5000D47130825006396E7003A
:1043D000130835002301B500139685004D8E139701
:1043E0000501518F3303F34093968501D98E1356FF
:1043F0002300AA97014794C305079107E36DC7FE01
:104400001377C3FFB307E8006307E3062380B70011
:1044100013871700637C1703A380B7001387270057
:10442000637617032381B700138737006370170380
:10443000A381B70013874700637A17012382B7006F
:104440001387570063741701A382B700828093F526
:10445000F50F13978500D98D139705014D8FE377DD
:1044600015FFAA87910723AEE7FEE3ED17FF8280D1
:1044700082802A8895B78280AA8749BF8347050032
:104480002A8799C7050583470500EDFF198D8280AE
:104490000145828005058347F5FF850503C7F5FFC4
:1044A00091C7E389E7FE3385E74082808147E5BF16
:1044B000AA87850503C7F5FF8507A38FE7FE75FB70
:1044C000828083460500930700026397F600050586
:1044D00083460500E38DF6FE938756FD93F7D70FCD
:1044E00085C7AA87814585CE01458507138606FDC8
:1044F0001317250083C607003A9506053295F5F691
:1045000099C13305A0408280938536FD834615000E
:1045100093B5150093071500E1FA0145D5B701459C
:1045200082809C412380A7009C4185079CC182809A
:1045300097C60100938606079C421757030013078E
:10454000672413861700BA972380A70097C5010038
:1045500023AAC504A9476308F5009307000463056F
:10456000F6000145828075DE370610F005078347A7
:10457000F7FF2320F6F09C42FD1797C5010023A307
:10458000F502EDF7014582804D712322911423201D
:104590002115232A511323248113232611142324A4
:1045A0008114232E3113232C411323286113232636
:1045B0007113232291132320A113232EB111AA8456
:1045C0002E8932C6130C5002A54A83470900638026
:1045D0008703B9CB804011A0A1CB2300F400804019
:1045E0000509050480C083470900E39787FF034658
:1045F000190093081900C686130D0002FD597D5A53
:104600000148130550059307D6FD93F7F70F13895B
:1046100016006363F52A17C701001307A79E8A07D0
:10462000BA979C43BA9782878320C11403248114CC
:1046300083244114032901148329C113032A8113FC
:10464000832A4113032B0113832BC112032C8112E4
:10465000832C4112032D0112832DC11171618280BF
:10466000A14C02C4854763D50715B2478040938BA0
:10467000770093F68BFF03AB060083A94600938770
:1046800086003EC6668681465A85CE85EF10D01DCF
:104690002AC8814763853723930D4101854B668680
:1046A00081465A85CE85EF10603E814666862A8B0C
:1046B000AE89EF10701BA24723A0AD0093861B00AC
:1046C000910D63843701B68BD9BFE37E9BFF63DD19
:1046D0004601A2872380A70180407D1A930714001A
:1046E0009CC03E84E3C846FF93962B001C08BE96F0
:1046F00031A8938777052300F4008040FD1B938742
:104700001B00050480C0F116E351F0EC9C42E3E28B
:10471000FAFE93870703C5B79C4093060003324710
:104720002380D7009C4093064700C14C1386170096
:1047300090C013068007A380C700804002C4BA87D8
:10474000050480C003AB0700814936C625BFB247C8
:1047500083AC0700938B470063840C1C635F401994
:104760009307D0026319FD1683C70C0085C363DC71
:1047700009189440850C7D1A2380F60080400504BA
:1047800080C083C70C00E5F7635D4001804093075C
:1047900000022300F40080407D1A050480C0E31A63
:1047A0000AFE5EC61DB502C48547A94CE3CF07EBE0
:1047B000B24780409386470071B703C61600CA8689
:1047C00099B59C40930650022380D7008040050491
:1047D00080C0E5BBC14C02C471B5B24703C6160028
:1047E000CA8683A9070091073EC6E35E0AE04E8AA7
:1047F000FD5911BD03C61600130DD002CA8621B59E
:104800009347FAFFFD8703C61600337AFA00CA867B
:10481000DDBB03C61600130D0003CA86EDB383C5C6
:104820001600930906FDCA86938705FD2E86E3EEE2
:10483000FAFA93972900BE9985068609AE9983C531
:104840000600938909FD938705FD2E86E3F3FAFEA2
:1048500069BF32479C40144311073AC62380D700F2
:104860008040050480C095B3854763D3070BB247EA
:1048700093867700E19A938786003EC683A9460017
:104880009C4263DC090A94401306D002B307F0404F
:104890002380C6008040B336F000B30930410504E0
:1048A00080C03E8BB389D940A94C02C4E1BB03C68A
:1048B00016000508CA8681BB9C40468921B7E37D66
:1048C0009BDD8547814B8546E3C547E131BD97CCEC
:1048D0000100938C2CAFCE856685EF007043330AC0
:1048E000AA40635C400180402300A40180407D1AFF
:1048F000050480C0E31A0AFE014A83C70C00E38264
:1049000007EAE3C809E6FD197D57E394E9E6ADBD82
:10491000B247938647009C4336C693D9F74195B773
:10492000635640019307D002E313FDFA97CC0100D0
:10493000938C4CA9930780021DBD3E8BA94C02C4E9
:10494000804089B34D71232E3113B70900409387FE
:10495000F9FF2324811423229114232C4113232AA9
:1049600051132326111423202115232861132326F4
:10497000711323248113232291132320A113232EA7
:10498000B1112A8A2EC417C401001304A4C1975A76
:104990000300938A2ADF97B401009384247C3EC6E7
:1049A00093055002294513080004B70610F0834709
:1049B0000A006386B704C1C71840050A130617002A
:1049C000569797C8010023AFC8BC2300F700638245
:1049D000A706E31E06FD175703001307A7DA05070E
:1049E0008347F7FF23A0F6F01C40FD1717C6010010
:1049F000232AF6BAEDF783470A00E39EB7FA834607
:104A00001A0013051A002A87930B00027D5B7D5C58
:104A1000014893055005A5489387D6FD93F7F70FF6
:104A2000130A170063E7F5348A07A6979C43A697F5
:104A30008287175703001307E7D455F28DBF8320F1
:104A4000C1140324811483244114032901148329EC
:104A5000C113032A8113832A4113032B0113832BD0
:104A6000C112032C8112832C4112032D0112832DBC
:104A7000C11171618280A14C014D854763DB07192B
:104A8000A2479D07E19B83AD070003AB4700138757
:104A900087003AC4668681466E85DA85EF10C05C71
:104AA0002AC863066D35130941018549668681462A
:104AB0006E85DA85EF00907D66868146AA8D2E8B05
:104AC000EF10805A2320A90085091109E3106DFF1A
:104AD000E3FE9DFD13060004B70610F063D18903C1
:104AE0001C4013871700D69797C5010023ACE5AA91
:104AF00023807701630CC7047D1CE3C389FFB247A1
:104B00006800A548B386F9008A061C08BE962948A5
:104B100013030004370610F0E384A6E89C429305D3
:104B2000000363F4F800930570051840AE979305F1
:104B30001700569717CE01002326BEA62300F700C4
:104B40006380072B638C6526F116F9B717570300AE
:104B5000130747C305078347F7FF23A0F6F01C4060
:104B6000FD1797C5010023AFF5A2EDF77D1C71B7C6
:104B70001C40130600041387170097C5010023A3E8
:104B8000E5A2B386FA00930500032380B600630F05
:104B9000C73C890797C6010023A6F6A0569793063F
:104BA00080072300D700175703001307A7BDB706D8
:104BB00010F0639EC70005078347F7FF23A0F6F0B8
:104BC0001C40FD1717C60100232EF69CEDF7A247E7
:104BD000C14C014D91072247014B832D07003EC474
:104BE00055BDA24783AC070013894700638E0C3A7A
:104BF000635480219307D002639EFB2E03C70C00F1
:104C0000BA856310072025AC8547A94C014DE3C93F
:104C100007E7A2479107C1B7A2478346170052870B
:104C200003AB070091073EC4E3580CDE5A8C7D5B52
:104C3000E5B383461700930BD0025287F1BB93472D
:104C4000FCFFFD8783461700337CFC005287E9B3E5
:104C500083461700930B000352877DBB0346170062
:104C6000138B06FD5287930706FDB286E3EEF8FA32
:104C700093172B00DA9705078607B29703460700BC
:104C8000138B07FD930706FDB286E3F3F8FE69BFB9
:104C9000A2451C402946984193861700D69717C510
:104CA00001002321D5902380E7001389450063008C
:104CB000C72A930700046387F6204AC4D5B1854705
:104CC00063DE0729A24713877700619B930787005C
:104CD0003EC4032B47001C43635A0B301840130695
:104CE00000049306170097C5010023ADD58A569797
:104CF0009305D0022300B7006387C62CB307F040AA
:104D00003337F000330B6041BE8D330BEB40A94CC1
:104D1000014D49B38346170005085287F5B983460C
:104D200017005287D5B91C4093060004138717005B
:104D300017C601002328E686D69713065002238063
:104D4000C700E31FD7C4175703001307A7A3B7066D
:104D500010F005078347F7FF23A0F6F01C40FD176E
:104D600017C601002320F684EDF71DB9C14C014D93
:104D700029B31C40930600042A8A1387170017C61C
:104D800001002321E682D697130650022380C70034
:104D9000E318D7C0175703001307C79EB70610F0D4
:104DA00005078347F7FF23A0F6F01C40FD1717B651
:104DB00001002329F67EEDF72A8ADDB61757030096
:104DC0001307479C05078347F7FF2320F6F01C4095
:104DD000FD1797B5010023A7F57CEDF7F1162DBB64
:104DE000175703001307079AF1FDF11635B3E3FCDB
:104DF0009DCB8549C5B1014C03C70C00BA85E30EB4
:104E000007EAFD58294513080004B70610F0635758
:104E10000B0A1C4013861700D69717B301002323F3
:104E2000C3782380E7006384A50663040609850C24
:104E300003C70C007D1CBA8579FBE35080E91C4058
:104E40009305000213060004B70610F021A07D1C94
:104E5000E3050CE613871700D6972380B70017B534
:104E600001002321E574BA87E313C7FE1757030037
:104E70001307479105078347F7FF23A0F6F01C406F
:104E8000FD1717B50100232FF570EDF7C9B71757B8
:104E900003001307278F41DE05078347F7FF23A091
:104EA000F6F01C40FD1717B60100232DF66EEDF746
:104EB000BDBF175703001307E78CF9BF7D1BE31A2B
:104EC0001BF5A5BF175703001307C78BB70610F0D4
:104ED00005078347F7FF23A0F6F01C40FD1717B620
:104EE00001002321F66CEDF74AC45DBC97BC0100BC
:104EF000938C4C4DDA856685212D330CAC40E35DF7
:104F000080EF1C4013060004B70610F021A07D1CA2
:104F1000E3030CEE13871700D6972380770197B52C
:104F2000010023A1E568BA87E313C7FE1757030002
:104F30001307478505078347F7FF23A0F6F01C40BA
:104F4000FD1797B5010023AFF564EDF7C9B7175703
:104F5000030013072783BDFA4AC499B4A2471387F5
:104F600047009C433AC413DBF741BDB31757030016
:104F700013074781B70610F005078347F7FF23A003
:104F8000F6F01C40FD1717B60100232DF660EDF773
:104F9000854717B701002327F76093078007174756
:104FA00003002301F77E25B1635680019307D002E9
:104FB000E39EFBF297BC0100938CCC401307800268
:104FC000930580023DBD974603009386A67B370676
:104FD00010F0850603C7F6FF2320E6F018407D1782
:104FE00097B5010023A0E55C6DF709BBBE8DA94C08
:104FF000014D4DB4B70710F023A0A7F201A03971FD
:10500000130341022ED29A8506CE32D436D63AD830
:105010003EDA42DC46DE1AC63532F24001452161F5
:1050200082805D711303810322D42AC632DC2A8474
:105030001A86680006D6BEC236DEBAC0C2C4C6C66C
:105040001ACEEFF06FD4B247238007003245B2503A
:10505000018D225461618280B70710F083A647F466
:1050600003A607F403A747F4E31AD7FE9306067DC9
:1050700033B6C600B305E60023A4D7F423A6B7F4DD
:105080008280B70710F003A747F403A607F483A6AE
:1050900047F4E31AD7FE9306067D33B6C60023A471
:1050A000D7F4B305E60023A6B7F49307000873A06E
:1050B00047308280411122C406C697B7010093870A
:1050C000E74E17B401001304244E98431C40930686
:1050D00047069387470617B601002327F64C8567D6
:1050E00017B601002324D64C938777BB63C6D7003D
:1050F000B240224441018280FD779387C74A3E97A0
:1051000097B7010023A4E74ACD2C85476310F50229
:1051100018408967938777320145E3DBE7FCEFF0BE
:105120007FED2244B24041016FC0FFED17B5010091
:105130001305C529EFF0BFEC0945EFF0BFEB2244A2
:10514000B24041016FC03FEC17B501001305C529FE
:105150006FF0FFEA17B50100130585296FF03FEAEC
:10516000411122C426C206C6856417B40100130487
:10517000A428938784380100FD17F5FF2285EFF0FE
:105180001FE8C5BF0945D9A8411106C6BD2405477A
:1051900081476316E500B2403E854101828017B524
:1051A00001001305A522EFF09FE5B24089473E8537
:1051B000410182807370043001A0828073700430DA
:1051C00001A0011122CC26CA4AC806CE2A84231780
:1051D00001000149854411A005495040084081461D
:1051E0009305E100EFB0FF90E31895FE631A090004
:1051F0001844835707008507C207C1872310F700AB
:105200008357E10085072317F100C1BF797122D4CC
:1052100026D24AD04ECE06D62A84814981440549F9
:105220005040084081469305E100EFB0DF9FE3194D
:1052300025FF8357E10063859700BE848549CDB77C
:105240008504639A09001844835707008507C2073D
:10525000C1872310F700C204C180D9B701114EC61F
:10526000AA89314506CE22CC26CA4AC8EFE03FEBD8
:105270002A84014689450545EFB04FC51309803E94
:1052800097B701009387473408C0232224011CC428
:105290003145EFE0DFE8AA8408404E87A28688C047
:1052A00017B501001305C53188C4814801488147FD
:1052B0001306004097B501009385451523A204000D
:1052C000170500001305C5F4EFC02FA9A686814875
:1052D0000148014781471306004097B501009385B7
:1052E000651317050000130505EEEFC00FA7314544
:1052F000EFE0FFE22A84014689450545EFB00FBD86
:1053000097B701009387E72B08C01CC42322040031
:105310003145EFE0DFE0AA840840A28623A2240101
:1053200088C017B501001305452A88C48148014883
:10533000814701471306004097B501009385050E8C
:10534000170500001305C5ECEFC02FA14E87A686F8
:105350008148014881471306004097B501009385B5
:10536000650C17050000130505E6EFC00F9F3145DA
:10537000EFE0FFDA2A84014689451545EFB00FB505
:1053800097B701009387072408C0232224011CC477
:105390003145EFE0DFD8AA840840A28623A2240189
:1053A00088C017B501001305652288C481480148EB
:1053B000814701471306004097B501009385050713
:1053C00017050000130525E0EFC02F996244F24055
:1053D0004249B249A686D2448148014881470147E3
:1053E0001306004097B501009385C504170500001A
:1053F000130505E205616FC04F9641114AC222C6EE
:1054000026C44EC017B501001305051C17B80100CE
:105410001308081B83540500835E050083590800A8
:1054200017B901001309C918035E080003542500C9
:105430008315090017B70100130707180353250048
:10544000831707008353280003162700C2098358D7
:10545000280093D9094183524500C2044204035FE6
:10546000450083162900835F4800C184B385354118
:10547000418403174700858F018EB335B000C20306
:1054800003154900B305B04093D30341B337F0008F
:105490003336C000C202ED8F3306C040B38676407B
:1054A00093D2024193950F01F18FB336D00003568A
:1054B000480033075740C1853244B306D0403337E4
:1054C000E0000D8D3307E040F58F3335A000F98FF4
:1054D0003305A04017B701002310D70F17B70100FD
:1054E0002318C70D17B701002319670C17B7010060
:1054F0002311170D17B701002312E70D17B701008D
:10550000231AC70AA244124982497D8D4101828033
:10551000B305B500930705006386B70003C707000E
:10552000631607003385A740678000009387170044
:105530006FF09FFE130101FB23229104232C4103F2
:1055400023229103232611042324810423202105EF
:10555000232E3103232A51032328610323267103B9
:10556000232481032320A103232EB101930C0500E2
:10557000138A05009304000063DE05003305A04094
:105580003337A000B305B040930C0500338AE540E3
:105590009304F0FF63DA06003306C040B337C0005F
:1055A000B306D040B386F640930A060093890600FE
:1055B00013840C0013090A006396062817BB010028
:1055C000130B4BCF6370CA16B70701006372F61452
:1055D0009307F00F63F4C70093098000B3573601B7
:1055E000330BFB0083470B0013050002B387370121
:1055F000B309F540638C0900B3153A01B3D7FC0039
:10560000B31A360133E9B70033943C0113DB0A01C6
:1056100093050B0013050900EF00507C130A0500E9
:1056200093050B00939B0A0113050900EF00907688
:1056300093DB0B019305050013850B00EF00D0727F
:10564000131A0A0193570401B367FA0063FAA7001B
:10565000B387570163E6570163F4A700B387570187
:105660003389A74093050B0013050900EF0010775D
:10567000130A050093050B0013050900EF00907154
:105680001314040193050500131A0A0113850B0076
:1056900013540401EF00506D33648A00637AA40050
:1056A00033045401636654016374A4003304540149
:1056B0003304A4403354340193050000638A04008A
:1056C00033048040B3378000B305B040B385F54064
:1056D000130504008320C1040324810483244104AE
:1056E000032901048329C103032A8103832A410377
:1056F000032B0103832BC102032C8102832C410263
:10570000032D0102832DC1011301010567800000F3
:10571000B707000193090001E362F6EC93098001E9
:105720006FF0DFEB631A060093050000130510000D
:10573000EF005066930A0500B707010063FAFA0EFE
:105740009307F00F63F4570193098000B3D73A0130
:10575000330BFB0083470B001305000233095A414A
:10576000B3873701B309F540E38209EAB39A3A01F6
:10577000335BFA00B3153A01B3D7FC0093DB0A019F
:1057800033E9B70013050B0093850B00EF0010659C
:10579000130A050093850B00139C0A0113050B00E7
:1057A000EF00505F135C0C019305050013050C001E
:1057B000EF00905B131A0A0193570901B367FA00CF
:1057C00033943C0163FAA700B387570163E657019E
:1057D00063F4A700B3875701338BA74093850B0071
:1057E00013050B00EF00905F130A050093850B0073
:1057F00013050B00EF00105A9305050013050C006C
:10580000EF00905693160901131A0A0193D6060168
:10581000B366DA0063FAA600B386560163E6560162
:1058200063F4A600B38656013389A6406FF01FDEED
:10583000B707000193090001E3EAFAF09309800138
:105840006FF0DFF06376DA0093050A006FF01FE770
:10585000B707010063FAF604930BF00F33B5DB00D2
:105860001315350033D7A60097B70100938787A497
:10587000B387E70083CB070093050002B38BAB002F
:10588000338B7541631C0B0263E4460163EACC0071
:105890003384CC40B306DA4033B98C0033892641D7
:1058A000930509006FF09FE1B707000113050001A0
:1058B000E3EAF6FA130580016FF0DFFAB3966601AA
:1058C000335D7601336DDD00B35D7A01B3156A0196
:1058D00033DC7C0113540D01336CBC0013850D00C7
:1058E00093050400B3196601EF00504F930A0500B9
:1058F0009305040013850D0033996C01931C0D0171
:10590000EF00504993DC0C01130A050093050500D4
:1059100013850C00EF005045939A0A0113570C01B0
:1059200033E7EA00930D0A00637EA7003307A7015F
:10593000930DFAFF6368A7016376A700930DEAFF52
:105940003307A701330AA7409305040013050A0093
:10595000EF00D04893050400930A050013050A00E0
:10596000EF005043930505001304050013850C0058
:10597000EF00903F93150C01939A0A0193D505010E
:10598000B3E5BA001307040063FEA500B385A501C3
:105990001307F4FF63E8A50163F6A5001307E4FF0E
:1059A000B385A501939D0D01B70C0100B3EDED008A
:1059B0001384FCFFB3F78D0033F48900338AA540CC
:1059C00013850700930504002326F10093DD0D01E4
:1059D000EF00903993050400930A050013850D002C
:1059E000EF00903813DC090193050C002324A1007B
:1059F00013850D00EF0050378327C10013040C00FE
:105A000093050400130C050013850700EF00D03543
:105A10008326810013D70A013305D5003307A70079
:105A20006374D700330C9C01B70701009387F7FF1D
:105A3000935507013377F70013170701B3F7FA00FF
:105A4000B3858501B307F7006366BA00631EBA0029
:105A5000637CF90033863741B3B7C700B385A541EE
:105A6000B385F54093070600B307F9403339F900D1
:105A7000B305BA40B385254133947501B3D76701A7
:105A80003364F400B3D565016FF05FC3130101FD0A
:105A900023229102232A5101232611022324810269
:105AA00023202103232E3101232C410123286101CE
:105AB0002326710123248101232291012320A101A6
:105AC000930A050093840500639E063813040600BC
:105AD0009309050017A901001309C97D63F8C512D0
:105AE000B7070100138B05006378F6101307F00F5A
:105AF0003337C70013173700B357E6003309F900EF
:105B0000834609003387E60093060002B386E64029
:105B1000638C0600B394D40033D7EA003314D60064
:105B2000336B9700B399DA00935A040193850A0006
:105B300013050B00EF00902A1309050093850A0056
:105B4000931B040113050B00EF00D02493DB0B0122
:105B5000930405009305050013850B00EF00D0208A
:105B60001319090193D70901B367F900138A0400D7
:105B700063FEA700B3878700138AF4FF63E88700FA
:105B800063F6A700138AE4FFB3878700B384A740B6
:105B900093850A0013850400EF00502413090500C3
:105BA00093850A0013850400EF00D01E9399090124
:105BB00093040500930505001319090113850B00D3
:105BC00093D90901EF00501AB36939011386040013
:105BD00063FCA900B30934011386F4FF63E689006E
:105BE00063F4A9001386E4FF13140A013364C400AC
:105BF000130A00006F000013B7070001130700012C
:105C0000E36CF6EE130780016FF01FEF138A0600B6
:105C1000631A06009305000013051000EF009017AB
:105C200013040500B7070100637EF4129307F00F19
:105C300063F48700130A8000B35744013309F90065
:105C4000034709009306000233074701B386E64085
:105C500063940612B3848440130A1000135B04019A
:105C600093050B0013850400EF005017130905007E
:105C700093050B0013850400931B0401EF009011A2
:105C800093DB0B01930405009305050013850B00BE
:105C9000EF00900D1319090193D70901B367F900BB
:105CA000938A040063FEA700B3878700938AF4FFFA
:105CB00063E8870063F6A700938AE4FFB387870051
:105CC000B384A74093050B0013850400EF00101167
:105CD0001309050093050B0013850400EF00900BDA
:105CE000939909019304050093050500131909010F
:105CF00013850B0093D90901EF001007B36939012F
:105D00001386040063FCA900B30934011386F4FF71
:105D100063E6890063F4A9001386E4FF13940A0183
:105D20003364C4001305040093050A008320C102F4
:105D30000324810283244102032901028329C10132
:105D4000032A8101832A4101032B0101832BC10016
:105D5000032C8100832C4100032D0100130101035A
:105D600067800000B7070001130A0001E366F4EC46
:105D7000130A80016FF05FEC3314D40033DAE400CF
:105D8000B399DA0033D7EA00935A0401B394D400EC
:105D900093850A0013050A00336B9700EF00100487
:105DA0001309050093850A0013050A00931B0401DB
:105DB000EF00407E93DB0B01930405009305050083
:105DC00013850B00EF00407A1319090113570B01DB
:105DD0003367E900138A0400637EA7003307870056
:105DE000138AF4FF636887006376A700138AE4FFD1
:105DF00033078700B304A74093850A001385040086
:105E0000EF00C07D1309050093850A001385040087
:105E1000EF004078930405009305050013850B00FF
:105E2000EF00807413170B011357070113190901B1
:105E3000B367E9001387040063FEA700B3878700F8
:105E40001387F4FF63E8870063F6A7001387E4FF76
:105E5000B3878700131A0A01B384A740336AEA00A4
:105E60006FF0DFDF63ECD51EB707010063F4F604C3
:105E70001307F00FB335D7009395350033D7B6002D
:105E800097A7010093870743B387E70003C707007D
:105E9000130A00023307B700330AEA4063160A0206
:105EA00013041000E3E096E833B6CA00134416006A
:105EB0006FF05FE7B707000193050001E3E0F6FC30
:105EC000930580016FF09FFBB35CE600B39646013B
:105ED000B3ECDC0033D4E40093DB0C01B397440152
:105EE00033D7EA0093850B0013050400336BF700EA
:105EF000B3194601EF00806E1309050093850B006E
:105F000013050400139C0C01EF00C068135C0C0126
:105F1000930405009305050013050C00EF00C06411
:105F20001319090113570B013367E90013840400A7
:105F3000637EA700330797011384F4FF636897011A
:105F40006376A7001384E4FF33079701B304A740E7
:105F500093850B0013850400EF00406813090500CA
:105F600093850B0013850400EF00C06293040500C5
:105F70009305050013050C00EF00005F93170B015C
:105F80001319090193D70701B367F90013860400B9
:105F900063FEA700B38797011386F4FF63E89701B8
:105FA00063F6A7001386E4FFB38797011314040177
:105FB000B70B01003364C4001389FBFF337D240158
:105FC00033F92901B384A7409305090013050D0097
:105FD000EF008059935C040193050900130B050041
:105FE00013850C00EF00405893D90901130C0500EC
:105FF0009385090013850C00EF0000571309050075
:106000009385090013050D00EF0000563305850147
:1060100093570B013385A700637485013309790118
:1060200093570501B387270163E6F402E392F4BCBA
:10603000B70701009387F7FF3375F50013150501C6
:10604000337BFB0033964A0133056501130A0000D8
:10605000E37AA6CC1304F4FF6FF09FB9130A000093
:10606000130400006FF01FCC130101FB23248104F3
:1060700023229104232E310323229103232611048A
:1060800023202105232C4103232A510323286103C4
:1060900023267103232481032320A103232EB1018E
:1060A000930C0500938905001304050093840500F3
:1060B000639E062613090600138A060097AA0100AC
:1060C000938A4A1F63F4C514B70701006376F6127A
:1060D0009307F00F63F4C700130A8000B35746011B
:1060E000B38AFA0003C70A00130500023307470109
:1060F000330AE540630C0A00B395490133D7EC003D
:1061000033194601B364B70033944C01935A090123
:1061100093850A0013850400EF00404C93090500A5
:1061200093850A00131B090113850400EF008046C4
:10613000135B0B019305050013050B00EF00C04234
:106140009399090193570401B3E7F90063FAA70093
:10615000B387270163E6270163F4A700B38727010C
:10616000B384A74093850A0013850400EF0000471D
:106170009309050093850A0013850400EF00804110
:1061800013140401930505009399090113050B00ED
:1061900013540401EF00403D33E48900637AA40006
:1061A00033042401636624016374A40033042401CE
:1061B0003304A44033554401930500008320C104F7
:1061C0000324810483244104032901048329C10396
:1061D000032A8103832A4103032B0103832BC1027A
:1061E000032C8102832C4102032D0102832DC10166
:1061F0001301010567800000B7070001130A0001C1
:10620000E36EF6EC130A80016FF05FED631A06008F
:106210009305000013051000EF00C03713090500B7
:10622000B7070100637AF90E9307F00F63F42701B3
:10623000130A8000B3574901B38AFA0003C70A0062
:1062400013050002B384294133074701330AE540AF
:10625000E30E0AEA33194901B3DAE900B3954901BB
:1062600033D7EC0093540901336BB70013850A0050
:1062700093850400EF0080369309050093850400A0
:10628000931B090113850A00EF00C03093DB0B015B
:106290009305050013850B00EF00002D939909016C
:1062A00093570B01B3E7F90033944C0163FAA7004D
:1062B000B387270163E6270163F4A700B3872701AB
:1062C000B38AA7409385040013850A00EF000031CC
:1062D000930905009385040013850A00EF00802BC5
:1062E0009305050013850B00EF00002893150B01A3
:1062F0009399090193D50501B3E5B90063FAA500A7
:10630000B385250163E6250163F4A500B385250166
:10631000B384A5406FF09FDFB7070001130A0001A7
:10632000E36AF9F0130A80016FF0DFF0E3E8D5E8E3
:10633000B707010063FCF604930BF00F33B5DB00E5
:106340001315350033D7A60097A70100938787F66A
:10635000B387E70083CB070093050002B38BAB0044
:10636000338B7541631E0B0263E4360163EACC0094
:106370003384CC40B386D94033B58C00B384A64077
:1063800013050400938504006FF05FE3B707000175
:1063900013050001E3E8F6FA130580016FF09FFA98
:1063A000B3966601335D7601336DDD0033D4790138
:1063B000B395690133DC7C0193540D01336CBC004F
:1063C0001305040093850400B31A6601EF00002151
:1063D000130A0500938504001305040033996C012A
:1063E000931C0D01EF00001B93DC0C01130405004E
:1063F0009305050013850C00EF000017131A0A011E
:1064000013570C013367EA00130A0400637EA700E8
:106410003307A701130AF4FF6368A7016376A70097
:10642000130AE4FF3307A701B309A74093850400CB
:1064300013850900EF00801A9385040013040500FA
:1064400013850900EF00001593050500930405006E
:1064500013850C00EF00401193150C011314040177
:1064600093D50501B365B4001387040063FEA5004E
:10647000B385A5011387F4FF63E8A50163F6A500C2
:106480001387E4FFB385A501131A0A01B70C0100B5
:10649000336AEA001384FCFFB3778A0033F48A007E
:1064A000B384A54013850700930504002326F1005B
:1064B000135A0A01EF00400B9309050093050400ED
:1064C00013050A00EF00400A13DC0A01930D0500D2
:1064D00093050C0013050A00EF0000098327C10093
:1064E000130A050093050C0013850700EF00C00791
:1064F0003305B50113D709013307A7006374B7014A
:10650000330A9A01B70701009387F7FF93550701F4
:106510003377F70013170701B3F7F900B385450187
:10652000B307F70063E6B400639EB400637CF90030
:1065300033865741B3B7C700B385A541B385F5404E
:1065400093070600B307F9403339F900B385B44027
:10655000B385254133947501B3D767013365F400E2
:10656000B3D565016FF09FC5130605001305000044
:1065700093F61500638406003305C50093D5150016
:1065800013161600E39605FE6780000063400506BB
:1065900063C6050613860500930505001305F0FF85
:1065A000630C060293061000637AB6006358C000BD
:1065B0001316160093961600E36AB6FE1305000044
:1065C00063E6C500B385C5403365D50093D6160094
:1065D00013561600E39606FE6780000093820000C3
:1065E000EFF05FFB13850500678002003305A040D4
:1065F00063D80500B305B0406FF0DFF9B305B040D4
:1066000093820000EFF01FF93305A040678002007D
:106610009382000063CA0500634C0500EFF09FF70A
:106620001385050067800200B305B040E35805FEFE
:106630003305A040EFF01FF63305B040678002003D
:10664000011122CC26CA2A84AE844AC84EC652C43E
:1066500056C206CEEFB03F9C1C4003290401B70987
:106660000001B3E59700930AC4000CC08144FD19F2
:10667000370A00021840638C2A03032609004A8562
:10668000B3654701B376360193175600758F03291A
:10669000490063C4070001E7F1BFE39DE6FC9317DF
:1066A000760063D30700D58CEFC09F84E1B793C415
:1066B000F4FFF98C04C0EFB01FBB0840F240624405
:1066C000D2444249B249224A924A0561828041112C
:1066D000094506C622C4EFE07FB817F7FFFF13078E
:1066E000A79D814605469305400617A501001305A1
:1066F00025D1EFD0EFD319C92A84EFB0DF922A86D3
:106700000147814685452285EFD02FDFEFB08FE925
:0A671000B24022440145410182809D
:02000004800278
:10000000BA47FEFFB848FEFFC247FEFFB848FEFFF2
:10001000B848FEFFB848FEFFB848FEFFDA47FEFFCB
:10002000B848FEFFB848FEFFF447FEFF0048FEFF59
:10003000B848FEFF1248FEFF1E48FEFF1E48FEFFA6
:100040001E48FEFF1E48FEFF1E48FEFF1E48FEFF24
:100050001E48FEFF1E48FEFF1E48FEFFB848FEFF7A
:10006000B848FEFFB848FEFFB848FEFFB848FEFF9C
:10007000B848FEFFB848FEFFB848FEFFB848FEFF8C
:10008000B848FEFFB848FEFFB848FEFFB848FEFF7C
:10009000B848FEFFB848FEFFB848FEFFB848FEFF6C
:1000A000B848FEFFB848FEFFB848FEFFB848FEFF5C
:1000B000B848FEFFB848FEFFB848FEFFB848FEFF4C
:1000C000B848FEFFB848FEFFB848FEFFB848FEFF3C
:1000D000B848FEFFB848FEFFB848FEFFB848FEFF2C
:1000E000B848FEFFB848FEFFB848FEFFB848FEFF1C
:1000F000B848FEFFB848FEFFB848FEFFB848FEFF0C
:100100005248FEFF6848FEFFB848FEFFB848FEFFB1
:10011000B848FEFFB848FEFFB848FEFFB848FEFFEB
:10012000B848FEFFAE48FEFFB848FEFFB848FEFFE5
:100130006046FEFF1847FEFFB848FEFFB848FEFFC6
:100140004E47FEFFB848FEFFA647FEFFB848FEFF39
:10015000B848FEFFD447FEFFC64BFEFF1A4CFEFF19
:10016000CE4BFEFF1A4CFEFF1A4CFEFF1A4CFEFF50
:100170001A4CFEFFC04AFEFF1A4CFEFF1A4CFEFF4F
:10018000DA4AFEFFE64AFEFF1A4CFEFFF84AFEFF7F
:10019000044BFEFF044BFEFF044BFEFF044BFEFF2F
:1001A000044BFEFF044BFEFF044BFEFF044BFEFF1F
:1001B000044BFEFF1A4CFEFF1A4CFEFF1A4CFEFFCA
:1001C0001A4CFEFF1A4CFEFF1A4CFEFF1A4CFEFFA3
:1001D0001A4CFEFF1A4CFEFF1A4CFEFF1A4CFEFF93
:1001E0001A4CFEFF1A4CFEFF1A4CFEFF1A4CFEFF83
:1001F0001A4CFEFF1A4CFEFF1A4CFEFF1A4CFEFF73
:100200001A4CFEFF1A4CFEFF1A4CFEFF1A4CFEFF62
:100210001A4CFEFF1A4CFEFF1A4CFEFF1A4CFEFF52
:100220001A4CFEFF1A4CFEFF1A4CFEFF1A4CFEFF42
:100230001A4CFEFF1A4CFEFF1A4CFEFF1A4CFEFF32
:100240001A4CFEFF1A4CFEFF1A4CFEFF1A4CFEFF22
:100250001A4CFEFF1A4CFEFF384BFEFF664BFEFFAA
:100260001A4CFEFF1A4CFEFF1A4CFEFF1A4CFEFF02
:100270001A4CFEFF1A4CFEFF1A4CFEFFBC4BFEFF51
:100280001A4CFEFF1A4CFEFF1E49FEFF184AFEFFE5
:100290001A4CFEFF1A4CFEFF8A4AFEFF1A4CFEFF64
:1002A000B04AFEFF1A4CFEFF1A4CFEFF144CFEFF34
:1002B000000102020303030304040404040404040D
:1002C00005050505050505050505050505050505DE
:1002D00006060606060606060606060606060606BE
:1002E00006060606060606060606060606060606AE
:1002F000070707070707070707070707070707078E
:10030000070707070707070707070707070707077D
:10031000070707070707070707070707070707076D
:10032000070707070707070707070707070707075D
:10033000080808080808080808080808080808083D
:10034000080808080808080808080808080808082D
:10035000080808080808080808080808080808081D
:10036000080808080808080808080808080808080D
:1003700008080808080808080808080808080808FD
:1003800008080808080808080808080808080808ED
:1003900008080808080808080808080808080808DD
:1003A00008080808080808080808080808080808CD
:1003B000546D725100000000546D7220537663003A
:1003C000286E756C6C2900004572726F7220696E20
:1003D00020416C74426C636B51207461736B7320A9
:1003E0000D0A00006D69616F750A00006D69616F2B
:1003F00075320A0068756E6772790A004368656332
:100400006B54696D6572000051436F6E7342310029
:100410005150726F644232005150726F6442330027
:1004200051436F6E734234005150726F6442350015
:0804300051436F6E7342360068
:100438001000000000000000017A5200017C010158
:100448001B0D02005000000018000000E050FEFFE5
:100458005805000000440E507489039406990B81D6
:1004680001880292049305950796089709980A9AB5
:100478000C9B0D036C010AC144C844C944D244D33F
:1004880044D444D544D644D744D844D944DA44DB88
:10049800440E00440B0000004C0000006C000000FB
:1004A800E455FEFFDC05000000440E30708903951A
:1004B8000781018802920493059406960897099883
:1004C8000A990B9A0C0370020AC144C844C944D261
:1004D80044D344D444D544D644D744D844D944DA40
:1004E800440E00440B00000050000000BC00000057
:1004F800705BFEFF0005000000440E5074880289FE
:10050800039305990B810192049406950796089721
:1005180009980A9A0C9B0D0320010AC144C844C9D2
:1005280044D244D344D444D544D644D744D844D9F7
:0C05380044DA44DB440E00440B000000D9
:0805CC00FC8F01000400000097
:040000058000004037
:00000001FF
